:100000000C9454040C947C040C947C040C947C0498
:100010000C947C040C947C040C947C040C947C0460
:100020000C947C040C947C040C947C040C947C0450
:100030000C947C040C947C040C947C040C947C0440
:100040000C947C1B0C947C040C947C040C947C0419
:100050000C947C040C947C040C947C040C947C0420
:100060000C94C61B0C947C04132C222C332C422C95
:10007000512C922C9E2C052CAD2C20202D2D204572
:10008000584954202D2D200053455454494E475370
:10009000202020200042414E44205343414E4E45F3
:1000A000522000534D415254205345415243480081
:1000B0004D414E55414C204D4F444500574F524BFA
:1000C000494E47204D4F444500202D2D204558498D
:1000D00054202D2D200043414C494252415445208B
:1000E00020200046494C5445523A4849474800466A
:1000F000494C5445523A4E4F524D414C0046494CA2
:100100005445523A4C4F5700554E4954533A206487
:10011000426D2000554E4954533A2025202020009E
:100120004155544F204C4F434B3A4F4646004155A2
:10013000544F204C4F434B3A4F4E0054494D4520AD
:1001400055503A34356D0054494D452055503A3399
:10015000306D0054494D452055503A31356D0054AD
:10016000494D452055503A4E4F4E452000414C4197
:10017000524D3A353025202000414C41524D3A3302
:100180003525202000414C41524D3A323025202067
:1001900000414C41524D3A4E4F4E45200007E01F62
:1001A000F8381C300C300CFFFFFC7FF93FF93FF8AA
:1001B0003FFC7FFEFFFEFFFEFFFFFFFFFFFE7C38E0
:1001C0001000000000E916D516C116AD1699168567
:1001D0001671165D16651678168B169E16B116C426
:1001E00016D716EA164916351621160D16FD1611E4
:1001F00017251739176C1680169416A816BC16D03A
:1002000016E416F8161A163F1664168916AE16D39B
:1002100016F8161D17F21417153C1561158615AB47
:1002200015D015F515B414A1A2A3A4A5A6A7A8B12D
:10023000B2B3B4B5B6B7B8E1E2E3E4E5E6E7E8F1B6
:10024000F2F3F4F5F6F7F8C1C2C3C4C5C6C7C8D106
:10025000D2D3D4D5D6D7D8FFBC00B000A300950028
:100260008800C9007A00D600C900FD00EF00E30055
:10027000140108012E0120015F01530147013B01D8
:100280009101850179016D01A1A2A3A4A5A6A7A84A
:10029000B1B2B3B4B5B6B7B8E1E2E3E4E5E6E7E896
:1002A000F1F2F3F4F5F6F7F8C1C2C3C4C5C6C7C886
:1002B000D1D2D3D4D5D6D7D8FFE916D516C116AD2D
:1002C000169916851671165D16651678168B169E8C
:1002D00016B116C416D716EA164916351621160D8C
:1002E00016FD161117251739176C1680169416A8C7
:1002F00016BC16D016E416F8161A163F16641689A0
:1003000016AE16D316F8161D17F21417153C156104
:10031000158615AB15D015F515B41428292A2B2CE4
:100320002D2E2F131220112110072208180609194B
:1003300005230A1A040B1B03240C1C020D1D2501A6
:100340000E1E000F1F261415271617300000000080
:10035000003E5B4F5B3E3E6B4F6B3E1C3E7C3E1C4B
:10036000183C7E3C181C577D571C1C5E7F5E1C0091
:10037000183C1800FFE7C3E7FF0018241800FFE748
:10038000DBE7FF30483A060E2629792926407F050B
:100390000507407F05253F5A3CE73C5A7F3E1C1C21
:1003A00008081C1C3E7F14227F22145F5F005F5FE1
:1003B00006097F017F006689956A606060606094CD
:1003C000A2FFA29408047E040810207E20100808D2
:1003D0002A1C08081C2A08081E101010100C1E0CDD
:1003E0001E0C30383E3830060E3E0E06000000006F
:1003F0000000005F00000007000700147F147F1456
:10040000242A7F2A1223130864623649562050009A
:1004100008070300001C2241000041221C002A1C86
:100420007F1C2A08083E0808008070300008080871
:100430000808000060600020100804023E51494591
:100440003E00427F400072494949462141494D33AF
:100450001814127F1027454545393C4A4949314116
:10046000211109073649494936464949291E0000E4
:100470001400000040340000000814224114141439
:100480001414004122140802015909063E415D5925
:100490004E7C1211127C7F494949363E414141222E
:1004A0007F4141413E7F494949417F090909013E58
:1004B000414151737F0808087F00417F410020407F
:1004C000413F017F081422417F404040407F021C91
:1004D000027F7F0408107F3E4141413E7F090909A8
:1004E000063E4151215E7F09192946264949493274
:1004F00003017F01033F4040403F1F2040201F3F3A
:100500004038403F631408146303047804036159BE
:10051000494D43007F414141020408102000414100
:10052000417F0402010204404040404000030708AC
:100530000020545478407F284444383844444428A8
:10054000384444287F385454541800087E0902184F
:10055000A4A49C787F0804047800447D40002040D7
:10056000403D007F1028440000417F40007C04781B
:1005700004787C080404783844444438FC18242463
:100580001818242418FC7C080404084854545424E3
:1005900004043F44243C4040207C1C2040201C3C60
:1005A0004030403C44281028444C9090907C446457
:1005B000544C4400083641000000770000004136EA
:1005C000080002010204023C2623263C1EA1A16170
:1005D000123A4040207A38545455592155557941A2
:1005E0002254547842215554784020545579400C77
:1005F0001E5272123955555559395454545939555A
:100600005454580000457C410002457D420001459C
:100610007C407D1211127DF0282528F07C54554530
:10062000002054547C547C0A097F4932494949329C
:100630003A4444443A324A4848303A4141217A3AAD
:1006400042402078009DA0A07D3D4242423D3D4079
:1006500040403D3C24FF2424487E4943662B2FFC28
:100660002F2BFF0929F620C0887E090320545479D6
:10067000410000447D413048484A32384040227AA7
:10068000007A0A0A727D0D19317D2629292F282624
:100690002929292630484D4020380808080808082C
:1006A0000808382F10C8ACBA2F102834FA00007B85
:1006B000000008142A142222142A14085500550098
:1006C00055AA55AA55AAFF55FF55FF000000FF0087
:1006D000101010FF00141414FF001010FF00FF1082
:1006E00010F010F0141414FC001414F700FF0000B4
:1006F000FF00FF1414F404FC141417101F10101F33
:10070000101F1414141F00101010F0000000001F20
:10071000101010101F10101010F010000000FF102B
:100720001010101010101010FF10000000FF140027
:1007300000FF00FF00001F10170000FC04F4141459
:100740001710171414F404F40000FF00F714141425
:1007500014141414F700F7141414171410101F10A5
:100760001F141414F4141010F010F000001F101FC8
:100770000000001F14000000FC140000F010F01036
:1007800010FF10FF141414FF141010101F000000AD
:1007900000F010FFFFFFFFFFF0F0F0F0F0FFFFFFB1
:1007A0000000000000FFFF0F0F0F0F0F3844443808
:1007B00044FC4A4A4A347E02020606027E027E0257
:1007C00063554941633844443C04407E201E200662
:1007D000027E020299A5E7A5991C2A492A1C4C729F
:1007E00001724C304A4D4D303048784830BC625A26
:1007F000463D3E494949007E0101017E2A2A2A2AB6
:100800002A44445F444440514A444040444A514091
:100810000000FF0103E080FF000008086B6B083652
:1008200012362436060F090F0600001818000000C3
:100830001010003040FF0101001F01011E00191DB2
:100840001712003C3C3C3C0000000000000000008F
:10085000240027002A0000000000250028002B00AB
:1008600000000000230026002900040404040404FE
:10087000040402020202020203030303030301024F
:10088000040810204080010204081020010204081E
:10089000102000000008000201000003040700000F
:1008A000000000000000183511241FBECFEFD8E073
:1008B000DEBFCDBF16E0A0E0B1E0E6E5F0E702C0A4
:1008C00005900D92A832B107D9F727E0A8E2B6E06B
:1008D00001C01D92A23CB207E1F714E0C4E5D4E0E8
:1008E00004C02197FE010E941738C335D107C9F70C
:1008F0000E9431210C9429380C9400006F927F9251
:100900008F929F92AF92BF92CF92DF92EF92FF921F
:100910000F931F93CF93DF93EC014B015A016901B1
:100920003801E881F9810284F385E02D870109957A
:10093000E881F981A501460D571D415051090284F6
:10094000F385E02D9601B401CE010995E881F98186
:100950000084F185E02D9301A501B401CE01099534
:10096000E881F981C80CD91CB60161507109008475
:10097000F185E02D9301A501CE010995DF91CF917D
:100980001F910F91FF90EF90DF90CF90BF90AF90AD
:100990009F908F907F906F9008952F923F924F92EB
:1009A0005F926F927F928F929F92AF92BF92CF92FF
:1009B000DF92EF92FF920F931F93CF93DF9300D0BC
:1009C0001F92CDB7DEB74C017B836A836A01590160
:1009D00017019801241B350B37FF03C03195219572
:1009E0003109C5014A815B81841B950B97FF03C0C8
:1009F00091958195910951E059838217930714F0DD
:100A000019820BC09A2D8B2D5801092F182F9A810E
:100A10008B81DB82CA82C92ED82E8A819B81A8163F
:100A2000B9065CF49C2D8D2D6801092F182F9A8131
:100A30008B81BB82AA82A92EB82E2501AA81BB81F7
:100A40004A1A5B0A38016C187D0877FE03C071945E
:100A500061947108720157FE03C0BFEFEB1AFB0AE5
:100A6000F594E794C016D1061CF00FEF1FEF1FC0DE
:100A700001E010E01CC0D401ED91FC91B98104802B
:100A8000F581E02D9101BB23C1F04A815B81B60164
:100A9000C4010995E618F708F7FE04C0C00ED11E80
:100AA000E40CF51CEA81FB813196FB83EA834A81E1
:100AB0005B81A416B506FCF604C0A6016A817B81A1
:100AC000E7CF0F900F900F90DF91CF911F910F9173
:100AD000FF90EF90DF90CF90BF90AF909F908F905E
:100AE0007F906F905F904F903F902F9008950F935D
:100AF0001F93CF93DF93DC0155968C9155978230ED
:100B000071F0833009F1813009F08CC01496ED91B9
:100B1000FC911597E41BF50BE21BF30B20C0149618
:100B2000ED91FC911597CF01861B970BBC0161508D
:100B300071091696ED91FC911797CF01841B950BC7
:100B4000AC01421B530B6EC01696ED91FC911797AA
:100B5000CF01861B970BBC0161507109FA0177FD2B
:100B60001BC116968D919C911797681779070CF009
:100B700013C1F7FF04C02E0F3F1FE0E0F0E0149612
:100B80008D919C911597AF01420F531F84179507C4
:100B90001CF49C012E1B3F0B121613060CF0FCC01C
:100BA000CB0177FD079643E0959587954A95E1F748
:100BB0009695982F882797958795E80FF91FE95EF6
:100BC000FE4F6770772781E090E001C0880F6A953B
:100BD000EAF7482F0130110541F088F00230110585
:100BE00009F0DAC02E0F3F1F15C02E0F3F1FE2176E
:100BF000F30709F4D1C08081842B8193F8CF8095CD
:100C00002E0F3F1FE217F30709F4C6C09081982307
:100C10009193F8CFE217F30709F4BEC080818427CF
:100C20008193F8CF77FDB8C014968D919C9115975C
:100C3000681779070CF0B0C057FF04C0240F351FA8
:100C400040E050E016968D919C911797FA01E20FC3
:100C5000F31F8E179F071CF49C01241B350B1216E3
:100C600013060CF099C0A22F842F86958695869541
:100C700090E8899F600D711D1124FB01E95EFE4F14
:100C80004770A9F198E0941B492F50E0EA01C05E3B
:100C9000DA4F8881291790F4421B51092FEF30E079
:100CA00002C0359527954A95E2F782230130110558
:100CB00041F068F00230110589F06EC00130110575
:100CC00019F42081822B0CC00130110520F480958D
:100CD0002081822305C00230110531F42081822752
:100CE0008083A91708F458C0A91BE058FF4FA8300B
:100CF00048F10230110559F4EF018A2F988190953F
:100D00009883C058DF4F88508830C0F730C081E0EA
:100D10000130110509F080E08195EF019A2F888359
:100D2000C058DF4F98509830D0F788EF8A0F8695DB
:100D30008695869590E8899FE00DF11D1124E05875
:100D4000FF4FA770AA2341F1B0E0A85EBA4F8C9183
:100D50000130110529F038F002301105D1F01CC026
:100D60009081892B18C080959081892314C088EFC9
:100D70008A0F86958695869590E8899FE00DF11DEE
:100D80001124E058FF4FA77039F0B0E0A85EBA4FC9
:100D90008C91908189278083DF91CF911F910F9152
:100DA00008950F931F93CF93DF93DC01FB015596BA
:100DB0008C915597823081F0833019F1813051F553
:100DC00014968D919C911597BC01641B750BAB011A
:100DD00041505109BF0181C014966D917C911597C6
:100DE000CB018E1B9F0BFC0116968D919C91179742
:100DF000BC01641B750BAB0141505109E21BF30BA5
:100E000009C016966D917C9117976E1B7F0B621B24
:100E1000730B63C057FD1CC116968D919C9117975B
:100E2000481759070CF014C1F7FF04C02E0F3F1FDD
:100E3000E0E0F0E014968D919C911597BF01620F50
:100E4000731F861797071CF49C012E1B3F0B12166D
:100E500013060CF0FDC0CA0157FD079663E0959597
:100E600087956A95E1F79695982F882797958795A6
:100E7000E80FF91FE95EFE4F4770552781E090E0CB
:100E800001C0880F4A95EAF7482F0130110541F05B
:100E900088F00230110509F0DBC02E0F3F1F15C08E
:100EA0002E0F3F1FE217F30709F4D2C08081842B75
:100EB0008193F8CF80952E0F3F1FE217F30709F4B7
:100EC000C7C0908198239193F8CFE217F30709F4F4
:100ED000BFC0808184278193F8CF57FDB9C0149695
:100EE0008D919C911597481759070CF0B1C077FF69
:100EF00004C0260F371F60E070E016968D919C911C
:100F00001797FB01E20FF31F8E179F071CF49C013C
:100F1000261B370B121613060CF09AC0A22F862F31
:100F200086958695869590E8899F400D511D1124E0
:100F3000FA01E95EFE4F6770A9F198E0961B492F10
:100F400050E0EA01C05EDA4F8881291790F4421B15
:100F500051092FEF30E002C0359527954A95E2F709
:100F600082230130110541F068F00230110589F04B
:100F70006FC00130110519F42081822B0CC00130A3
:100F8000110520F480952081822305C002301105CF
:100F900031F4208182278083A91708F459C0A91B46
:100FA000E058FF4FA83048F10230110559F4EF0125
:100FB0008A2F988190959883C058DF4F8850883049
:100FC000C0F731C081E00130110509F080E0819562
:100FD000EF019A2F8883C058DF4F98509830D0F790
:100FE00088EF8A0F86958695869560E8869FE00D46
:100FF000F11D1124E058FF4FA770AA2349F1B0E07A
:10100000A85EBA4F8C910130110529F038F00230FA
:101010001105D9F01DC09081892B03C08095908166
:101020008923808315C088EF8A0F869586958695DB
:1010300070E8879FE00DF11D1124E058FF4FA77065
:1010400039F0B0E0A85EBA4F8C9190818927E9CF42
:10105000DF91CF911F910F910895FC0177FD9AC008
:1010600080859185681779070CF094C057FD92C070
:1010700082859385481759070CF08CC0858982308A
:1010800009F07CC084819581DC01A61BB70BBD01F2
:101090006150710986819781FC01E41BF50BAF015A
:1010A000415051090AC0813041F484819581841BEB
:1010B000950BAB01BC01615071092130310529F05C
:1010C00008F122303105E1F10895FA0157FD379614
:1010D000A3E0F595E795AA95E1F7F695FE2FEE27A3
:1010E000F795E7956E0F7F1FFB01E95EFE4F477096
:1010F000552781E090E001C0880F4A95EAF790817A
:10110000892B3AC0FA0157FD379623E0F595E7950C
:101110002A95E1F7F695FE2FEE27F795E7956E0FE6
:101120007F1FFB01E95EFE4F4770552781E090E08D
:1011300001C0880F4A95EAF78095908189231CC0E9
:10114000FA0157FD379683E0F595E7958A95E1F723
:10115000F695FE2FEE27F795E7956E0F7F1FFB01A3
:10116000E95EFE4F4770552781E090E001C0880F8F
:101170004A95EAF79081892780830895833009F0A2
:1011800092CF86819781861B970BBA01AC014150A3
:10119000510993CF08950F931F93683823E1720785
:1011A0008105910568F0DC01CB01813727E19207C9
:1011B000A105B10548F080E797E1A0E0B0E004C0E8
:1011C00088E893E1A0E0B0E08F5D9140A109B1090A
:1011D0008C019D0146E036952795179507954A9510
:1011E000D1F78F739927AA27BB27B695A79597950F
:1011F000879567E0000F111F221F331F6A95D1F7F3
:10120000BC01CD01600F711F821F931F1F910F91B1
:1012100008950C9469350C946135CF92DF92EF926A
:10122000FF92CF938F3248F4E82FF0E0EE0FFF1FCC
:10123000E754FD4F6591749124C08091A907082E51
:10124000000C990BC09724E6289FB001299F700DD0
:10125000112468577C4E8091AA07082E000C990B28
:10126000C0974AE0489F9001499F300D1124620FBA
:10127000731F8091AB07082E000C990BC097680F65
:10128000791F80E090E00E94CB086B01E12CF12CEB
:1012900095E0CC0CDD1CEE1CFF1C9A95D1F781E18A
:1012A000C82A60E08FE00E94AD1A60E080E10E94F1
:1012B000AD1AC9E1C0FE02C061E001C060E081E199
:1012C0000E94AD1A61E08FE00E94AD1A60E08FE0ED
:1012D0000E94AD1AF694E794D794C794C15051F781
:1012E00061E080E10E94AD1A60E081E1CF91FF9062
:1012F000EF90DF90CF900C94AD1A4F925F926F9267
:101300007F928F929F92AF92BF92CF92DF92EF9295
:10131000FF920F931F93CF93DF9386EF91E00E948C
:101320000B0980932C06109232061092310610920F
:10133000300610922F0600E485E10E94191BEC0193
:1013400084E10E94191B20913106309132062C0F46
:101350003D1F3093320620933106C0912F06D09165
:1013600030068C0F9D1F9093300680932F060150FE
:1013700019F746E0359527954A95E1F7EC0156E0D7
:10138000D595C7955A95E1F780911601873061F59B
:1013900080910E0190910F012817390720F43093A6
:1013A0000F0120930E0180910C0190910D01821785
:1013B000930720F430930D0120930C0180910601D6
:1013C00090910701C817D90720F4D0930701C09363
:1013D000060180910401909105018C179D0720F46E
:1013E000D0930501C0930401C0901201D090130165
:1013F000E12CF12CC901330FAA0BBB0B9C01AD01F1
:101400002C193D094E095F09A7ECB0E00E94963502
:1014100020911001309111014901A12CB12CA5019D
:1014200094012C193D094E095F090E947735690125
:101430007A018FEFC81AD80AE80AF80A80900A01E0
:1014400090900B01A12CB12CCE01DD0FAA0BBB0B90
:101450009C01AD01281939094A095B09A7ECB0E0E4
:101460000E94963520910801309109012901612CD3
:10147000712CA3019201281939094A095B090E94BC
:101480007735BA01A9014F5F5F4F6F4F7F4FCA0198
:101490001C141D0444F429ECC216D1043CF038ECB1
:1014A000C32ED12C03C0CC24C394D12CD0923206AD
:1014B000C0923106181619063CF4EA01493C510560
:1014C0002CF0C8ECD0E002C0C1E0D0E0D0933006F0
:1014D000C0932F06CC15DD0514F4FC2C01C0FC2EA6
:1014E00000910101013021F0023019F41C2F01C0DC
:1014F0001C2D6F2D70E080E090E00E94E7364B01DC
:101500005C01612F70E080E090E00E94E736A50169
:1015100094010E94D235A50194010E943F3620E03B
:1015200030E048EC52E40E947A374B015C0120E045
:1015300030E0A9010E94753718161CF4C501B401EA
:1015400003C0C501B40190580E94B13662307105E4
:10155000C4F01F1520F0C02F1092770618C090918C
:1015600077069F5F96305CF0109277068F2D90E0A3
:101570008C159D0541F08C179D0719F406C09093BA
:101580007706C02F04C0C1E004C0C2E009C001302A
:1015900039F461E085E00E94AD1A60E086E006C0A3
:1015A00061E086E00E94AD1A60E085E00E94AD1A1D
:1015B000C0930101C13021F080911601873029F4D8
:1015C000809131069091320604C080912F0690914F
:1015D00030061816190634F4893C91052CF088EC75
:1015E00090E002C081E090E0DF91CF911F910F91D8
:1015F000FF90EF90DF90CF90BF90AF909F908F9033
:101600007F906F905F904F9008950E94701B209183
:10161000280630912906621B730B6E31710550F458
:101620008EE190E09C01261B370BB90180E090E031
:101630000C94361B0895982FEBE1F3E080E02491A1
:10164000291729F08F5F31968033C9F780E008951C
:10165000CF92DF92EF92FF921F93CF93DF93EC0133
:1016600061E08EE00E94AD1A10E087E0E82EF12CD8
:101670009FEBC92E97E0D92E812F90E08C179D0704
:1016800080F461E084E00E94AD1AC7010197F1F790
:1016900060E084E00E94AD1AC6010197F1F71F5F78
:1016A000EBCF60E08EE00E94AD1A60E084E00E9423
:1016B000AD1ABE0180E090E0DF91CF911F91FF90C5
:1016C000EF90DF90CF900C94361B0F931F93CF9326
:1016D000DF9380911601863009F48CC0893009F0BF
:1016E0007FC080910201823008F470C0609138069A
:1016F00081E090E00E9409096091150180E090E08E
:101700000E94090984EF91E00E940B098093020175
:1017100040913806C0E090E02C2F30E0821793070C
:101720005CF0F901E754F84F2081421303C0C093E5
:10173000370608C0CF5FF0CF80910201813099F069
:10174000815011C080910201C817B0F70C2F10E032
:10175000C80146960E940B09682FC80145960E9451
:101760000909CF5FEFCF809302016091020184EFFE
:1017700091E00E94090960E08EE190E00E94090971
:1017800009EB17E0C5E1D0E0CE010E940B09F8019A
:1017900081938F012196CE31D105B1F78091380622
:1017A000E82FEE0FFF0BE754FD4F6591749141E078
:1017B0000E948D1DC5E082E390E00E94280BC1507D
:1017C000D1F7809102018093370603C080E00E9428
:1017D0009B12809115018093160181E08093390658
:1017E0006CED75E080E090E0DF91CF911F910F915B
:1017F0000C94361B6091380681E090E00E94090944
:101800006091150180E090E00E9409099091020129
:101810006091380680E0492F50E0282F30E04217D1
:1018200053070CF479C0F901E754F84F208162178F
:10183000A1F08F5FF2CF809102018F5F893008F0B5
:1018400088E0809302018091020190E06091380667
:1018500045960E94090980910201809337066091A4
:1018600037068EE190E00E94090909EB17E0C5E117
:10187000D0E0CE010E940B09F80181938F012196DF
:10188000CD31D105B1F76091020184EF91E00E9462
:10189000090980913806E82FEE0FFF0BE754FD4F42
:1018A00065917491803339F52091A907022E000CBF
:1018B000330B2053310994E6929FB001939F700D32
:1018C000112468577C4E2091AA07022E000C330B7E
:1018D000205331099AE0929FA001939F500D11244B
:1018E000640F751F2091AB07022E000C330B2053A1
:1018F0003109620F731F40E00E948D1DC5E082E335
:1019000090E00E94280BC150D1F7809115018330DF
:1019100009F061CF82E05FCF983009F08CCFC1E051
:1019200080910201C81708F086CF0C2F10E0C80183
:1019300046960E940B09682FC80145960E94090926
:10194000CF5FEECF1F93CF93DF9382E390E00E94AF
:10195000280B60912E0680E00E94F41C89E00E9412
:10196000841A892BD9F3C0E016E0D8E0C13029F001
:10197000C23011F1C11103C01FC010931601609154
:101980002E068C2F0E94F41C89E00E94841A892B59
:10199000B1F080912E068111E9CF88E00E94841A6F
:1019A000892B51F5C15084E690E00E94280BC3308A
:1019B000A4F5C7FFDBCFC2E0D0931601E0CF89E0EA
:1019C0000E94841A892B21F08091150180931601C1
:1019D00084E690E00E94280B64E670E080E090E0EE
:1019E0000E94361BC1111BC090912E0681E08927F1
:1019F00080932E06C5E007C08AE00E94841A892BD6
:101A000049F4CF5FD0CF82E390E00E94280BC15011
:101A1000D1F705C0C3300CF4A9CFC0E0CDCFDF9122
:101A2000CF911F910895CF92DF92FF920F931F9352
:101A3000CF93DF931092170561E08EE00E94DD1ACC
:101A400061E084E00E94DD1A60E084E00E94AD1A4B
:101A500060E088E00E94DD1A62E088E00E94AD1A32
:101A600060E089E00E94DD1A62E089E00E94AD1A20
:101A700060E08AE00E94DD1A62E08AE00E94AD1A0E
:101A800060E08BE00E94DD1A62E08BE00E94AD1AFC
:101A900060E08CE00E94DD1A62E08CE00E94AD1AEA
:101AA00060E08DE00E94DD1A62E08DE00E94AD1AD8
:101AB00061E085E00E94DD1A61E086E00E94DD1AA7
:101AC00061E080E10E94DD1A61E081E10E94DD1A9F
:101AD00061E08FE00E94DD1A60E085E10E94DD1A7E
:101AE00060E084E10E94DD1A82E08093E9068CE3E5
:101AF0008093E8068091EA068F3F09F4BDC061E05B
:101B00008091EC060E94DD1A61E08091EE060E9451
:101B1000DD1A8091EE06082E000C990BFC01E659A7
:101B2000F74FE491F0E0EE0FFF1FEA5AF74F2591CF
:101B300034913093F5062093F406FC01E258F74FF8
:101B4000E491E093FA068091EC06082E000C990BC4
:101B5000FC01E659F74FE491F0E0EE0FFF1FEA5A5F
:101B6000F74F259134913093F7062093F606FC0148
:101B7000E258F74FE491E093FB068091EF06811164
:101B80003EC061E08091EA060E94DD1A61E080912A
:101B9000EB060E94DD1A8091EB06082E000C990BD3
:101BA000FC01E659F74FE491F0E0EE0FFF1FEA5A0F
:101BB000F74F259134913093F3062093F206FC0100
:101BC000E258F74FE491E093F9068091EA06082E77
:101BD000000C990BFC01E659F74FE491F0E0EE0F91
:101BE000FF1FEA5AF74F259134913093F106209365
:101BF000F006FC01E258F74FE491E093F80680917B
:101C0000EF06882309F45FC0CFB7F894809175067A
:101C1000811127C0E4E7F8E08491E8E8F8E09491C6
:101C2000E82FF0E0EE0FFF1FE45BF74FA591B491B2
:101C3000EC91E92321F461E08AE00E94AD1A61E0B1
:101C40008AE00E94DD1A8CB580618CBD8CB5806401
:101C50008CBD61E08DE00E94DD1A61E08BE00E94A6
:101C6000DD1A809175068F5F80937506CFBF80E582
:101C70008CBD81E08DBD27C0109258071092570788
:101C80001092A0061092C10610929E0681E08093E9
:101C90009D061092780661E082E10E94AD1A61E033
:101CA00083E10E94AD1A8091B9008E7F8093B900C4
:101CB0008091B9008D7F8093B90088E48093B8004B
:101CC00085E48093BC008091ED0687FD1EC061E035
:101CD0000E94DD1A61E08091ED060E94AD1A61E07C
:101CE00070E080E090E00E94361B60E08091ED069D
:101CF0000E94AD1A6AE070E080E090E00E94361B1E
:101D000061E08091ED060E94AD1A8EEA0E942711D3
:101D100085ED0E94271180E80E94271188EA0E9421
:101D200027118FE30E94271183ED0E94271180E085
:101D30000E94271180E40E9427118DE80E9427113C
:101D400084E10E94271180E20E94271180E00E9416
:101D5000271181EA0E94271188EC0E9427118AED41
:101D60000E94271182E10E94271181E80E94271119
:101D70008FEC0E94271189ED0E94271181EF0E94AC
:101D800027118BED0E94271180E40E94271184EA1D
:101D90000E94271186EA0E9427118EE20E942711D5
:101DA0008FEA0E9427110E94701160ED77E080E0B9
:101DB00090E00E94361B84E690E00E940B0985317A
:101DC00009F49BC0833109F489C060EA82E090E0A5
:101DD0000E94090960E083E090E00E9409096EE535
:101DE00084E090E00E94090961E085E090E00E94B3
:101DF000090960EA87E090E00E94090960E088E054
:101E000090E00E9409096EE589E090E00E940909CE
:101E100061E08AE090E00E94090963E080E090E0E0
:101E20000E94090960E081E090E00E94090965E7ED
:101E300075E08FEA97E00E9422380FEA17E0C5E6C6
:101E4000D0E0F80161918F01CE010E94090921962D
:101E5000CE36D105B1F76DE775E089EA97E00E94CB
:101E6000223809EA17E0C2E7D1E0F80161918F0159
:101E7000CE010E9409092196C837F1E0DF07A9F7D2
:101E800060E08FE190E00E94090960E08EE190E05F
:101E90000E94090960E385E190E00E940909C6E11A
:101EA000D0E06C2F665FCE010E9409092196CE31E9
:101EB000D105B9F760E088EF91E00E94090960E080
:101EC00087EF91E00E94090968E084EF91E00E94A9
:101ED000090961E086EF91E00E94090960E08AEF5C
:101EE00091E00E94090960E089EF91E00E940909F0
:101EF00065E184E690E00E9409098EE190E00E948D
:101F00000B09F82E809337068FE190E00E940B09B1
:101F1000182F8093760686EF91E00E940B0980933C
:101F20002C0687EF91E00E940B098093340688EF1E
:101F300091E00E940B09809336068AEF91E00E949F
:101F40000B098093350684EF91E00E940B09082F5E
:101F50008093020186EF91E00E940B0980932C068A
:101F600089EF91E00E940B098093330679EBC72E2D
:101F700077E0D72EC5E1D0E0CE010E940B09F60133
:101F800081936F012196CE31D105B1F70F1518F469
:101F900081E080933706183010F01092760688E0C2
:101FA000809316018091370690E045960E940B09B8
:101FB0008093380680932D060FEA17E0C5E6D0E03F
:101FC000CE010E940B09F80181938F012196CE3634
:101FD000D105B1F709EA17E0C2E7D1E0CE010E94CE
:101FE0000B09F80181938F012196C837F1E0DF07D3
:101FF000A9F785E090E00E940B09C82F84E090E0EB
:102000000E940B092C2F30E0322F2227282B3093EF
:1020100011012093100183E090E00E940B09C82F6A
:1020200082E090E00E940B092C2F30E0322F222713
:10203000282B309313012093120188E090E00E9436
:102040000B09C82F87E090E00E940B092C2F30E08D
:10205000322F2227282B30930B0120930A018AE08C
:1020600090E00E940B09C82F89E090E00E940B09C4
:102070002C2F30E0322F2227282B30930901209378
:102080000801C1E0C09339060E94701B60933A06B4
:1020900070933B0680933C0690933D0661E08EE092
:1020A0000E94AD1A809138060E940D0961E085E01A
:1020B0000E94AD1A60E086E00E94AD1AC093010153
:1020C00060E08EE0DF91CF911F910F91FF90DF9044
:1020D000CF900C94AD1ACF938BE00E94841AC1E08C
:1020E000019709F0C0E08CE00E94841A019709F47E
:1020F000CE5F8DE00E94841A019709F4CC5F8C2F8B
:10210000CF9108952091C10690915607213208F091
:102110004AC080919E068111FCCF32E030939E062A
:1021200031E030939D063FEF30939C0610929B0662
:1021300020939A06A1EAB6E04AE756E0FA013E2F5C
:10214000341B321718F43D913193F9CF1092790670
:1021500020917906990F922B9093790690917806A9
:10216000913061F410927806909179069093BB00BB
:102170009091BC0093FDF8CF95EC01C095EE909343
:10218000BC0090919E069230E1F390919C069F3F97
:1021900079F080919C06803241F080919C068033DA
:1021A00031F084E005C081E003C082E001C083E03B
:1021B0001092A0061092C10610929F060895909169
:1021C000EF06992339F08EBD00000DB407FEFDCF58
:1021D0008EB5089528E030E040E8E091F206F091F5
:1021E000F30650819091F906909595239083E091A4
:1021F000F006F091F1069091F806542F582319F04B
:102200005081952B03C05081909595239083E09148
:10221000F206F091F30650819091F906952B908388
:10222000469521503109C9F60895009769F0FC01DF
:1022300001900020E9F73197AF01481B590BBC0111
:102240008EEC96E00C94541680E090E00895CF93C5
:10225000C82F8091EA068F3F59F1E091F406F09182
:10226000F50680819091FA06982B9083E091F6060E
:10227000F091F70620819091FB0690959223908330
:10228000E091F406F091F50620819091FA06909580
:10229000922390838C2F0E94DF10E091F406F0913E
:1022A000F50690818091FA06892B8083CF9108955D
:1022B0008091E80691E090939F06809356071092D4
:1022C000A0061092C10660E082EC96E00E945517CD
:1022D0006C2F82EC96E00E945517CF910C948210DF
:1022E000EF92FF920F931F93CF93DF9381E20E94AF
:1022F000271180E00E9427118FE70E94271182E2B8
:102300000E94271180E00E94271187E00E94271178
:102310008091EA068F3F79F1E091F406F091F5069D
:1023200090818091FA06892B8083E091F606F091E6
:10233000F70690818091FB06892B8083E091F4065B
:10234000F091F50690818091FA068095892380832B
:10235000C7E1D1E089910E94DF1085E0C731D8073D
:10236000C9F7E091F406F091F50690818091FA06A4
:10237000892B808330C0F090B8008CE08093B80047
:10238000C7E1D1E0EE24E3948091E806E0929F0655
:10239000809356071092A0061092C10660E482EC6A
:1023A00096E00E94551700E010E0FE01E00FF11FDB
:1023B000608182EC96E00E9455170F5F1F4F00313D
:1023C000110599F70E948210609685E0C731D80701
:1023D000D9F6F092B800DF91CF911F910F91FF9045
:1023E000EF9008950C9415112F923F924F925F92A7
:1023F0006F927F928F929F92AF92BF92CF92DF9215
:10240000EF92FF920F931F93CF93DF9300D000D0F2
:10241000CDB7DEB7E22FF0E0FC83EB83442E512CE6
:10242000262E312C682E712C8F01041915090E5F90
:102430001F4F9101261937092E5F3F4FA2014150CE
:102440005109B30161507109E12CF12C8EEC96E039
:102450000E94201AC10102979A838983430192E066
:10246000890E911CEE24E394F12C820129813A819A
:10247000A201B4018EEC96E00E94CD040B811C8178
:1024800029813A81A801B4018EEC96E00E94CD0426
:10249000CB80DC80E2E0CE1AD1085201F2E0AF0E30
:1024A000B11C86019301A501B3018EEC96E00E9458
:1024B000CD049101A501B1018EEC96E00E94CD04FE
:1024C00082019401A501B3018EEC96E00E94CD0437
:1024D0000B811C819401A601B3018EEC96E00E9451
:1024E000CD0485019101A20169817A818EEC96E08B
:1024F0000E94CD04860191014B815C8169817A81C2
:102500008EEC96E00E94CD040F900F900F900F90EC
:10251000DF91CF911F910F91FF90EF90DF90CF90BF
:10252000BF90AF909F908F907F906F905F904F90F3
:102530003F902F900895CF93C82F2CE244E168E696
:1025400088E10E94F41181E090E09093DF0680938F
:10255000DE061092E1061092E0068AE190E0909388
:10256000DB068093DA0688E190E09093DD068093A5
:10257000DC06CC2319F081E995E002C084E895E0FF
:102580000E94F2118AE190E09093DB068093DA06D4
:1025900082E290E09093DD068093DC06CC2319F074
:1025A00083EA95E002C08EE995E00E94F211CF9196
:1025B0000C9470118F929F92AF92BF920F931F93C2
:1025C000CF93DF93CDB7DEB7A1970FB6F894DEBFF8
:1025D0000FBECDBF19A2423008F44AE08E010F5D54
:1025E0001F4F842E912CA12CB12CA50194010E9487
:1025F000A135E62FB901CA0101501109EA3014F4DE
:10260000E05D01C0E95CD801EC93232B242B252B42
:1026100061F7C8010E941511A1960FB6F894DEBFAC
:102620000FBECDBFDF91CF911F910F91BF90AF90A3
:102630009F908F900895BC0180E090E04AE00C9458
:10264000DA12E091CE06F091CF060190F081E02DF4
:10265000682F8EEC96E00994CF92DF92EF92FF9272
:10266000CF93DF936C01990FEE08FF08F7FE17C0B8
:102670008DE20E942113EC0166277727CB016C19AC
:102680007D098E099F094AE00E94DA128C0F9D1F76
:10269000DF91CF91FF90EF90DF90CF9008954AE0C7
:1026A000C701B601DF91CF91FF90EF90DF90CF90FF
:1026B0000C94DA123F924F925F926F927F928F92B8
:1026C0009F92AF92BF92CF92DF92EF92FF920F93C1
:1026D0001F93CF93DF93D82FC62FD42E322E4801CD
:1026E000BE2C80910107481709F47DC0D13009F450
:1026F000A6C08E2D90E0A0E0B0E09C01AD0121507D
:10270000310941095109A7E0B0E00E94963527EC54
:1027100030E040E050E00E94773529013A018FEF28
:10272000481A580A680A780A60910407462F4695A5
:1027300046954695677009E010E0041915098BE08D
:10274000489FA00111244150510988E0689FB001C1
:102750001124625C7F4FE12CF12C23E030E08EEC01
:1027600096E00E94201A60910407462F46954695F0
:10277000469567708BE0489FA0011124475F5F4F2B
:102780004419550988E0689FB0011124625C7F4FAD
:10279000EE24E394F12C820123E030E08EEC96E00D
:1027A0000E94201A80EA8B15F0F0D330E1F460919A
:1027B0000407462F46954695469567708BE0489FDF
:1027C000A001112488E0689FB0011124625C7F4F52
:1027D000E12CF12C08E010E023E030E08EEC96E0F4
:1027E0000E94201A2CC0AA2061F1D230D1F581E0DC
:1027F00090E09093E1068093E0069093DF0680934B
:10280000DE0686E090E09093DB068093DA068AE0AD
:1028100090E09093DD068093DC060E94701B24EF0D
:1028200031E040E050E00E94A1356A3F710581052A
:10283000910548F48BEA95E00E94F21112C0A110B4
:1028400010C0D23071F4E12CF12C0AE010E020E24B
:1028500030E04AE050E065E070E08EEC96E00E94E7
:10286000201AD0920107C0930407E12CF12C00E458
:1028700010E02EE230E044E150E060E070E08EECE9
:1028800096E00E94201A84E08093E20681E090E0C6
:102890009093E1068093E0069093DF068093DE0636
:1028A00082E090E09093DB068093DA0684E190E08A
:1028B0009093DD068093DC068C2F8770D82EC8326B
:1028C00040F46C2D70E080E090E040E10E94DA126C
:1028D00008C08CE40E9421138D2D90E001960E9487
:1028E0002C1382E08093E20601E010E01093E106F1
:1028F0000093E0061093DF060093DE061092DB06DD
:102900001092DA0682E390E09093DD068093DC0675
:10291000C4010E941B131093E1060093E00610937C
:10292000DF060093DE0681E08093E206C83040F4C3
:102930001092DF061092DE06EE24E394F12C06C01E
:102940001092E1061092E006E12CF12C0AE010E072
:1029500028E030E040E050E060E370E08EEC96E08C
:102960000E94201A81E390E09093DB068093DA06C0
:1029700001E010E01093DD060093DC0682E595E0AF
:102980000E94F21188EF8C0F883060F41092DF06FD
:102990001092DE061093E1060093E006EE24E39425
:1029A000F12C0AC01093DF060093DE061092E106B8
:1029B0001092E006E12CF12C0AE010E028E030E073
:1029C0004BE050E060E370E08EEC96E00E94201A4D
:1029D00081E390E09093DB068093DA068CE090E050
:1029E0009093DD068093DC0680E595E00E94F2116D
:1029F00080EF8C0F883070F41092DF061092DE06A4
:102A000081E090E09093E1068093E006EE24E39469
:102A1000F12C0CC081E090E09093DF068093DE06FD
:102A20001092E1061092E006E12CF12C0AE010E091
:102A300028E030E046E150E060E370E08EEC96E0A4
:102A40000E94201A81E390E09093DB068093DA06DF
:102A500087E190E09093DD068093DC068DEF95E0B2
:102A60000E94F21188EE8C0F883070F41092DF060D
:102A70001092DE0681E090E09093E1068093E006FC
:102A8000EE24E394F12C0CC081E090E09093DF06FB
:102A90008093DE061092E1061092E006E12CF12C04
:102AA0000AE010E028E030E041E250E060E370E04E
:102AB0008EEC96E00E94201A81E390E09093DB0672
:102AC0008093DA0682E290E09093DD068093DC0644
:102AD00081EB95E00E94F21180EE8C0F883070F44B
:102AE0001092DF061092DE0681E090E09093E106FE
:102AF0008093E006EE24E394F12C0CC081E090E09A
:102B00009093DF068093DE061092E1061092E006B5
:102B1000E12CF12C0AE010E028E030E04CE250E03B
:102B200060E370E08EEC96E00E94201A81E390E072
:102B30009093DB068093DA068DE290E09093DD06B9
:102B40008093DC0683EB95E00E94F211C83270F0AE
:102B50001092DF061092DE0681E090E09093E1068D
:102B60008093E006EE24E394F12C0CC081E090E029
:102B70009093DF068093DE061092E1061092E00645
:102B8000E12CF12C0AE010E028E030E047E350E0CF
:102B900060E370E08EEC96E00E94201A81E390E002
:102BA0009093DB068093DA0688E390E09093DD064D
:102BB0008093DC0681E695E00E94F211832D90E07F
:102BC000A0E0B0E09C01AD0121503109410951095B
:102BD000A7E0B0E00E94963527EC30E040E050E0FE
:102BE0000E94773529013A018FEF481A580A680A7E
:102BF000780AC695C695C6958BE0C89FE00111245A
:102C00005E0181E0A81AB10888E0D89E6001112415
:102C10008EE3C80ED11C09E010E004191509E12C5F
:102C2000F12C23E030E0A501B6018EEC96E00E9485
:102C3000201A2996AE0144195509EE24E394F12C8B
:102C4000820123E030E0B6018EEC96E00E94201A6B
:102C50000E94701B24EF31E040E050E00E94A1355B
:102C6000663971058105910560F4E12CF12C09E0CC
:102C700010E023E030E0A501B6018EEC96E00E9462
:102C8000201ADF91CF911F910F91FF90EF90DF906D
:102C9000CF90BF90AF909F908F907F906F905F90FC
:102CA0004F903F900C947011CF92DF92EF92FF9271
:102CB0000F931F93CF93DF936C017A018B01C0E0D8
:102CC000D0E0CE15DF0589F0D8016D918D01D601D8
:102CD000ED91FC910190F081E02DC6010995892BC1
:102CE00011F47E0102C02196ECCFC701DF91CF9194
:102CF0001F910F91FF90EF90DF90CF900895833058
:102D000081F028F4813099F08230A1F00895873065
:102D1000A9F08830B9F08430D1F4809180008F7DA3
:102D200003C0809180008F7780938000089584B5E0
:102D30008F7702C084B58F7D84BD08958091B000E7
:102D40008F7703C08091B0008F7D8093B00008958D
:102D50003FB7F8948091A5079091A607A091A70787
:102D6000B091A80726B5A89B05C02F3F19F0019682
:102D7000A11DB11D3FBFBA2FA92F982F8827820F01
:102D8000911DA11DB11DBC01CD0142E0660F771F51
:102D9000881F991F4A95D1F7089585ED8093BC004F
:102DA0008091BC0084FDFCCF10929E060895409156
:102DB0007B07262F30E0240F311D21323105DCF452
:102DC00020919E062430C9F4FC0180E090E0861733
:102DD00058F430917B072191DC01A75AB84FA30F1B
:102DE000B11D2C930196F3CF80917B07680F609300
:102DF0007B0780E0089581E0089582E008950895BA
:102E000081E090E03091580720915707321710F475
:102E100080E090E0919581959109089580915807FF
:102E200090915707891730F48F5F8093580780E09F
:102E300090E008958FEF9FEF08958091570790E0FD
:102E400020915807821B91090895CF92DF92EF924B
:102E5000FF920F931F93CF93DF937C01262F972F21
:102E60008A0180919F06882391F0C62FD72F6E018B
:102E7000C40ED51ECC15DD0571F06991D701ED9119
:102E8000FC910190F081E02DC7010995F3CF642FEB
:102E9000822F0E94D716C801DF91CF911F910F9109
:102EA000FF90EF90DF90CF900895CF93DF931F9224
:102EB000CDB7DEB7698320919F062223D1F0209100
:102EC000C106203240F021E030E0FC013383228350
:102ED00080E090E015C08091A006E82FF0E0EF556B
:102EE000F94F998190838F5F8093A0068093C106EC
:102EF00005C061E0CE0101960E94D71681E090E006
:102F00000F90DF91CF91089508952F923F924F92A5
:102F10005F926F927F928F929F92AF92BF92CF9269
:102F2000DF92EF92FF920F931F93CF93DF93CDB772
:102F3000DEB76B970FB6F894DEBF0FBECDBF4C0166
:102F40005A8349831F830E83FD82EC82CB82DC018E
:102F500058964D915C9159974115510509F0A5C0BE
:102F600018968D919C911997681779070CF05AC1A2
:102F70001A968D919C911B97E981FA81E817F907C0
:102F80000CF050C1D12CCB013B81F6E03F9F800D6E
:102F9000911D1124181619060CF044C1C60133E026
:102FA000880F991F3A95E1F749815A81840F951F3F
:102FB000181619060CF036C157968C91811103C072
:102FC000203B08F02F5F55E0259F900111247E875C
:102FD0006D875B01212CC901861B970B9987888718
:102FE000A981BA811896BB87AA87B5E02B1641F054
:102FF000E885F985EA0DFB1DE45BFC4F349001C0C8
:10300000312C69807A80230130FE12C0D401ED9109
:10301000FC91BB81B13031F40480F581E02D2E812B
:103020003F8118C00684F785E02DEE80FF801CC02C
:10303000EC81FD812E813F81E217F307E1F0D4019D
:10304000ED91FC91BB81B13051F40480F581E02D0C
:103050002C813D81A301B501C40109950CC00684F2
:10306000F785E02DEC80FD8086019601A2016D853B
:103070007E85C40109953694EFEF6E1A7E0A4C0CDA
:103080005D1C2A853B856216730609F0BDCF23942B
:103090003FEFA31AB30A4D855E854C0D5D1D5E871B
:1030A0004D8756E02512A1CFBDC0FA013496349168
:1030B000329785919491231BA7E02A9F800D911D43
:1030C0001124FA01259134913A8B298BFC0125902A
:1030D0003490FC01329634913887319644914C8774
:1030E0003196E491FC013596A491319684915B81EF
:1030F000523050F06A2E0A2E000C7708E82F082E66
:10310000000CFF0BFB87EA87FB81CF2ED12C6C9C38
:1031100090016D9C300D7C9C300D1124A901460F4F
:10312000571F588B4F871C82A12CEA2FAA0FFF0B29
:103130003B016E0E7F1E5885650F711DDB01AE0FC2
:10314000BF1FBF8BAE8BE981FA81E80FF11D87FDB0
:10315000FA95F98FE88F9C85A91608F063C08A2D2F
:1031600090E04A855B85480F591F4C9D90014D9D0D
:10317000300D5C9D300D1124A981BA81A20FB31FBF
:10318000BE87AD877B8E6A8E4F845888BC81B61906
:10319000BB8BE88DF98DE80FF91FFD8BEC8B8B89CC
:1031A000FA8D8F0F2A8D3B8D4E895F892417350745
:1031B00099F1877041F4C1010196E989FA89E20D1C
:1031C000F31DB4901C01B7FE1EC0D401ED91FC911B
:1031D000BB81B13061F40480F581E02D2E813F8107
:1031E0004C895D896A8D7B8DC40109950CC006846C
:1031F000F785E02DEE80FF80860196014D855E8586
:10320000B201C4010995BB0CEA8DFB8D3196FB8F91
:10321000EA8F4C0C5D1CC3CF5C818885580F5C83A2
:10322000A39499CF6B960FB6F894DEBF0FBECDBFB7
:10323000DF91CF911F910F91FF90EF90DF90CF9092
:10324000BF90AF909F908F907F906F905F904F90C6
:103250003F902F900895AF92BF92CF92EF92FF923E
:103260000F931F93CF93DF93EC01262F888D998DB9
:10327000009709F042C06A3069F42C898E859F85D9
:1032800038E0239F800D911D11249F878E871D8616
:103290001C86ACC06D3009F4A9C08E898823C1F0AA
:1032A0003C898C859D8546E0349F800D911D1124BD
:1032B00048855985841795075CF01D861C868E8588
:1032C0009F85E8E03E9F800D911D11249F878E878A
:1032D000EA88FB88088919894E855F856C857D851C
:1032E000CC88CE010E9485172C898C859D85F6E0BF
:1032F0002F9F800D911D112441C06A3079F41D86E5
:103300001C862C89FC013696E4918E859F852E9F24
:10331000800D911D11249F878E8768C06D3009F440
:1033200065C0AC014C5F5F4FFA013491631708F43C
:103330005DC03196E491E61708F458C0FA01449153
:10334000362F341BFC013296A590B490F7E03F9FD6
:10335000A00CB11C1124F501329634913196E49100
:10336000332311F0E1110DC0F5013496E4912C895D
:103370008C859D85E29F800D911D11249D878C87F2
:1033800035C0F501359644915E89552311F16C895C
:10339000E32FF0E0E40FF11D47FDFA956E9FD00199
:1033A0006F9FB00D11244C855D854A0F5B1FE8852A
:1033B000F9854E175F076CF01D861C86FC0136965A
:1033C000E4918E859F856E9F800D911D11249F87AE
:1033D0008E87EA88FB88088919894E855F856C8508
:1033E0007D85CC88CE010E948517BECF81E090E01C
:1033F000DF91CF911F910F91FF90EF90CF90BF90F1
:10340000AF900895EF92FF920F931F93DC01ED911F
:10341000FC9111971A960D911C911B9718962D915E
:103420003C9119970684F785E02D7B0140E050E040
:1034300060E070E009951F910F91FF90EF90089563
:103440006F927F928F929F92AF92BF92CF92DF92B4
:10345000EF92FF920F931F93CF93DF936C015A016A
:103460004801EB013B01620E731EC615D70574F4CB
:10347000D601ED91FC910084F185E02D8701940146
:10348000A501BE01C60109952196EFCFDF91CF912D
:103490001F910F91FF90EF90DF90CF90BF90AF9072
:1034A0009F908F907F906F900895EF92FF920F936F
:1034B0001F93DC01ED91FC91260F371F215031093C
:1034C0000680F781E02D78018A0109951F910F91FF
:1034D000FF90EF900895EF92FF920F931F93780162
:1034E000DC01ED91FC91240F351F89010150110978
:1034F0000680F781E02D9B0109951F910F91FF90A8
:10350000EF9008950E941D38CF93DF93282F30E06D
:10351000F901EE56F74F8491F901E258F74FD49133
:10352000F901E659F74FC491CC2391F081110E9423
:103530007F16EC2FF0E0EE0FFF1FE05AF74FA5913A
:10354000B491EC91ED2381E090E021F480E002C0A1
:1035500080E090E0DF91CF9108951F93CF93DF93A8
:10356000282F30E0F901EE56F74F8491F901E25827
:10357000F74FD491F901E659F74FC491CC23C9F024
:10358000162F81110E947F16EC2FF0E0EE0FFF1F27
:10359000EA5AF74FA591B4918FB7F894111105C06D
:1035A0009C91ED2FE095E92302C0EC91ED2BEC937B
:1035B0008FBFDF91CF911F910895CF93DF9390E05C
:1035C000FC01E258F74F2491FC01E659F74F849132
:1035D000882361F190E0880F991FFC01E45BF74FAD
:1035E000C591D491FC01EA5AF74FA591B4916111AC
:1035F00009C09FB7F8948881209582238883EC9135
:103600002E230BC0623061F49FB7F8943881822F6B
:10361000809583238883EC912E2B2C939FBF06C02B
:103620008FB7F894E8812E2B28838FBFDF91CF913D
:1036300008958E3008F08E5087702091170590E421
:10364000299F90011124822B80937C0080917A0025
:10365000806480937A0080917A0086FDFCCF80910F
:1036600078002091790090E0922B08958F929F929C
:10367000AF92BF92CF92DF92EF92FF926B017C01EB
:103680000E94A8164B015C01C114D104E104F104AD
:10369000F1F00E94A816DC01CB0188199909AA094A
:1036A000BB09883E9340A105B10570F321E0C21A21
:1036B000D108E108F10888EE880E83E0981EA11C6D
:1036C000B11CC114D104E104F10419F7DDCFFF905E
:1036D000EF90DF90CF90BF90AF909F908F90089524
:1036E0002FB7F8946091A1077091A2078091A3076A
:1036F0009091A4072FBF08951F920F920FB60F92BB
:1037000011242F933F938F939F93AF93BF938091F7
:10371000A1079091A207A091A307B091A4073091AF
:10372000A00723E0230F2D3720F40196A11DB11D22
:1037300005C026E8230F0296A11DB11D2093A00706
:103740008093A1079093A207A093A307B093A40727
:103750008091A5079091A607A091A707B091A8070F
:103760000196A11DB11D8093A5079093A607A09374
:10377000A707B093A807BF91AF919F918F913F91F9
:103780002F910F900FBE0F901F9018951F920F92C0
:103790000FB60F9211242F933F934F935F936F9324
:1037A0007F938F939F93AF93BF93EF93FF938091FA
:1037B000B900887F803609F49CC068F5883209F426
:1037C0005BC090F4803109F454C038F4882309F4C4
:1037D000F6C0883009F44DC0F6C0883109F44CC0F9
:1037E000803209F45DC0EFC0803409F468C048F449
:1037F000803309F455C0883309F0E5C080939C06F6
:10380000D8C0803509F44FC0883509F45DC08834CC
:1038100009F0D9C0D6C0883909F4C7C0A8F48837E0
:1038200009F467C038F4883609F463C0803709F4B6
:1038300060C0C9C0883809F4B8C0803909F45FC0D5
:10384000803809F0C0C05BC0803B09F486C038F402
:10385000803A09F466C0883A09F47FC0B4C0803C5D
:1038600009F4A7C0883C09F4A4C0883B09F48AC0C5
:10387000AAC08091790610C090919B0680919A060B
:10388000981770F5E0919B0681E08E0F80939B0660
:10389000F0E0E658F94F80818093BB0085EC86C04C
:1038A00080939C068EC0E0919B0681E08E0F8093F2
:1038B0009B068091BB00F0E0E658F94F8083909121
:1038C0009B0680919A066EC0E0919B0681E08E0F68
:1038D00080939B068091BB00F0E0E658F94F80830F
:1038E00080919D0681116DC081E08093780684EA05
:1038F00061C083E080939E0610929F07CFCF809196
:103900009F07803208F051C0E0919F0781E08E0F41
:1039100080939F078091BB00F0E0E158F84F8083CF
:10392000BDCF85EC8093BC0010929E0680919F07CE
:10393000803230F4E0919F07F0E0E158F84F1082B8
:1039400060919F0770E0E0917D07F0917E078FE71F
:1039500097E0099510929F0736C084E080939E06F9
:1039600010927C0710927B07E0917907F0917A071B
:10397000099580917B07811105C081E080937B07C9
:1039800010925907E0917C0781E08E0F80937C07AD
:10399000F0E0E75AF84F80818093BB0090917C075C
:1039A00080917B07981708F479CF85E88093BC0055
:1039B0000AC085EC8093BC0010929E0604C0109251
:1039C0009C060E94CD16FF91EF91BF91AF919F9100
:1039D0008F917F916F915F914F913F912F910F90B8
:1039E0000FBE0F901F901895EF92FF920F931F93A9
:1039F000CF93DF93D82FC62F611103C021E34FE08F
:103A000002C027E249E165E58CE20E94F4118AE0F8
:103A1000D89FA0011124C11103C04F5E5F4F02C0A7
:103A2000455E5F4FEE24E394F12C0AE010E026E2BD
:103A300030E06EE270E08EEC96E00E94201A81E0A9
:103A400090E0D11102C080E090E09093E106809375
:103A5000E0069093DF068093DE06CC2319F08CE11C
:103A600090E002C082E190E02FE230E03093DB068C
:103A70002093DA069093DD068093DC06CC2319F0C0
:103A80008BEB95E002C085EB95E00E94F211C1112D
:103A90003CC081E090E0D13011F480E090E0909360
:103AA000E1068093E0069093DF068093DE068FE2C6
:103AB00090E09093DB068093DA068CE190E090939F
:103AC000DD068093DC0682EC95E00E94F21181E035
:103AD00090E0D23011F480E090E09093E106809382
:103AE000E0069093DF068093DE0685E390E09093F6
:103AF000DB068093DA0686E290E09093DD06809301
:103B0000DC0686E096E00E94F211DF91CF911F91D2
:103B10000F91FF90EF900C947011CF92DF92EF9283
:103B2000FF920F931F93CF93DF93C82F6B01D42F76
:103B300021E34FE063E68EE10E94F411EE24E3946A
:103B4000F12C0AE010E022E430E041E150E060E2D4
:103B500070E08EEC96E00E94201A1092E10610921E
:103B6000E0061092DF061092DE06D1110FC084E34A
:103B700090E09093DB068093DA0682E190E09093E8
:103B8000DD068093DC0689EC95E00EC08EE290E0C5
:103B90009093DB068093DA0682E190E09093DD0655
:103BA0008093DC068AE895E00E94F21181E090E0C3
:103BB0009093E1068093E0069093DF068093DE0603
:103BC00005E210E01093DB060093DA0686E290E04F
:103BD0009093DD068093DC068EEC95E00E94F21156
:103BE0001093DB060093DA068CE190E09093DD06FB
:103BF0008093DC06C03321F1C83218F081E695E0ED
:103C000016C0C03218F083EB95E011C0C83118F02F
:103C100081EB95E00CC0C03118F08DEF95E007C046
:103C2000C83018F080E595E002C082E595E00E947A
:103C3000F211C7708C2F90E001960E942C1308C0DF
:103C40008091AD070E9421138091AE070E9421133D
:103C500087EC95E00E94F211C6010E941B1388EDCB
:103C600095E00E94F211DF91CF911F910F91FF908B
:103C7000EF90DF90CF900C947011EF92FF920F9322
:103C80001F93CF93C82F21E34FE065E58CE20E949C
:103C9000F4118AE0C89FA00111244F5E5F4FEE240B
:103CA000E394F12C0AE010E026E230E06EE270E0EE
:103CB0008EEC96E00E94201A81E090E0C11102C0D3
:103CC00080E090E09093E1068093E0069093DF0619
:103CD0008093DE0685E390E09093DB068093DA061E
:103CE00082E190E09093DD068093DC0689EC95E01C
:103CF0000E94F21181E090E0C13011F480E090E088
:103D00009093E1068093E0069093DF068093DE06B1
:103D10008FE290E09093DB068093DA068CE190E0EE
:103D20009093DD068093DC068AE895E00E94F2110C
:103D300081E090E0C23011F480E090E09093E106E1
:103D40008093E0069093DF068093DE0685E390E0A3
:103D50009093DB068093DA0686E290E09093DD068E
:103D60008093DC0686E096E00E94F211CF911F91CD
:103D70000F91FF90EF900C94701180E094E0E7E1D8
:103D8000F1E0DF019C011D9221503040E1F7EEECA3
:103D9000F6E081E0848B81E090E0938B828B918BC5
:103DA000808B0895EF92FF920F931F93CF93DF9331
:103DB0000E94BD1EECEFF6E0118284E6848312823D
:103DC00013821186CEECD6E04A855B854B505109B3
:103DD00028853985EE24E394F12C8A0160E070E0B7
:103DE000CE010E94CD040A851B850B50110928E1E4
:103DF00030E040E050E068E170E0CE010E94CD0488
:103E00008A859B8509971D861C869F878E878CEDEA
:103E100095E00E94F2118A859B85099728E330E09E
:103E20003D872C879F878E8781EE95E00E94F21157
:103E30008A859B850997288539852C5131093D87CD
:103E40002C879F878E8786EE95E00E94F2111D8653
:103E50001C860CE010E01F870E878BEE95E00E9419
:103E6000F21184E690E09D878C871F870E87DF9193
:103E7000CF911F910F91FF90EF900C947011EF92E2
:103E8000FF920F931F93CF93C82F7B018A012EE0DF
:103E900040E064E78CE00E94F41121E030E03093D0
:103EA000E1062093E0063093DF062093DE062091A2
:103EB000D6063091D706205631093695279530938E
:103EC000DB062093DA0684E090E09093DD06809391
:103ED000DC068EEC95E00E94F211C7010E941B13D4
:103EE00080EF95E00E94F211C8010E941B1322E3AB
:103EF00041E168E688E10E94F4118AE0C89FA001D0
:103F000011244D5E5F4FEE24E394F12C0AE010E0A3
:103F10002DE430E06AE170E08EEC96E00E94201A19
:103F200081E090E0C11102C080E090E09093E10652
:103F30008093E0069093DF068093DE062091D606FC
:103F40003091D70628543109369527953093DB06F2
:103F50002093DA0685E190E09093DD068093DC06FD
:103F600082EF95E00E94F21181E090E0C13011F4FF
:103F700080E090E09093E1068093E0069093DF0666
:103F80008093DE062091D6063091D706225431095F
:103F9000369527953093DB062093DA068FE190E083
:103FA0009093DD068093DC068FEF95E00E94F2117E
:103FB00081E090E0C23011F480E090E09093E1065F
:103FC0008093E0069093DF068093DE068091D6060C
:103FD0009091D7064897969587959093DB068093A6
:103FE000DA0689E290E09093DD068093DC0686E0B5
:103FF00096E00E94F211CF911F910F91FF90EF90E8
:104000000C9470112F923F925F926F927F928F92D9
:104010009F92AF92BF92CF92DF92EF92FF920F9357
:104020001F93CF93DF9300D000D000D0CDB7DEB781
:104030003C016B015A0179011801C901079697FDEE
:1040400007969C0193E0359527959A95E1F73A8379
:104050002983812C912C00E010E0021513050CF04F
:1040600043C01E821D82D801AC0DBD1DBC83AB8335
:10407000ED81FE81EE15FF0584F58D819E818770AF
:104080009927892B11F0550C0EC0ED81FE81F7FDAB
:10409000379683E0F595E7958A95E1F7E80DF91DE8
:1040A000EA0DFB1D549057FE12C0E091CE06F09130
:1040B000CF060480F581E02D21E030E04B815C816A
:1040C0006D817E81660D771D8EEC96E009958D8160
:1040D0009E8101969E838D83CBCF0F5F1F4F2981D9
:1040E0003A81820E931EB9CF26960FB6F894DEBFA2
:1040F0000FBECDBFDF91CF911F910F91FF90EF9039
:10410000DF90CF90BF90AF909F908F907F906F90F7
:104110005F903F902F9008955F926F927F928F9261
:104120009F92AF92BF92CF92DF92EF92FF920F9346
:104130001F93CF93DF93982E562E8FEF8093010716
:104140000E94BD1E81E090E09093E1068093E0061E
:104150009093DF068093DE0698120DC082E090E017
:104160009093DB068093DA061092DD061092DC064F
:104170008BE096E02FC082E098120DC086E090E0C0
:104180009093DB068093DA061092DD061092DC062F
:1041900083E196E01FC083E098121EC088E090E0A3
:1041A0009093DB068093DA061092DD061092DC060F
:1041B0008AE196E00E94F21186E090E09093DB069F
:1041C0008093DA068AE090E09093DD068093DC0627
:1041D00080E296E00E94F211A12CB12C98E0C92E49
:1041E000D12C3501CFE3D0E0812C81E0981209C0B9
:1041F000E82DF0E0E754F84F808190E086159705B0
:1042000059F4EE24E394F12C86019E01A601BE012F
:104210008EEC96E00E94CD048394581430F78FEF13
:10422000681A780A2896CF37D105F1F68BE0C80EC8
:10423000D11C88E0A80EB11C80E3A816B10489F651
:10424000DF91CF911F910F91FF90EF90DF90CF9072
:10425000BF90AF909F908F907F906F905F900C94E5
:104260007011CF93DF93CDB7DEB76F970FB6F89489
:10427000DEBF0FBECDBF789484B5826084BD84B5A7
:10428000816084BD85B5826085BD85B5816085BD51
:1042900080916E00816080936E0010928100809109
:1042A0008100826080938100809181008160809391
:1042B0008100809180008160809380008091B100B6
:1042C00084608093B1008091B00081608093B000E1
:1042D00080917A00846080937A0080917A00826075
:1042E00080937A0080917A00816080937A00809137
:1042F0007A00806880937A001092C1000E94130DAA
:1043000089E00E94841A892B09F05AC00E94701B10
:1043100060933A0670933B0680933C0690933D066B
:10432000109116018FEF810F843018F425E02D8352
:1043300002C031E03D8384E690E00E94280B1982A0
:1043400089E00E94841A892B69F459815A3051F00E
:1043500064E670E080E090E00E94361B49814F5F88
:104360004983EECF111103C083E0809316013324FB
:1043700033947FE0272EE2E64E2EE2E05E2EF8E553
:10438000CF2EF2E0DF2EAAE5AA2EA2E0BA2EBEE5DD
:104390008B2EB2E09B2E1CE5612E12E0712E8981DE
:1043A0008A3010F40C94942D80911601813011F014
:1043B0000C948C2D8AE0809316018FEF809314016A
:1043C000109272069091390680911601911105C0E4
:1043D00090911401891709F46CC01092390683304A
:1043E00019F128F4813069F1823041F15EC08630E4
:1043F00009F459C0873011F40C94212F843009F04E
:1044000054C08093150110927006EBE1F3E0E49143
:10441000E093380610926F0610926E0681E080934A
:104420006D060E94D21E41C090E590930301109248
:104430006F0610926E0691E09093740660910201EF
:104440002BC009EB17E095E1E92EF12CC7010E9482
:104450000B09D8018D938D01BFEFEB1AFB0AEEE13A
:10446000EE16F10499F78EE190E00E940B0981119C
:1044700001C081E0809337068091370690E0459631
:104480000E940B098093380684EF91E00E940B098B
:1044900080930201682F81E00E948C208091160198
:1044A0008093150102C00E94650B809116018093D4
:1044B000140110911601183009F00FC10E946B1001
:1044C0000E946B108F8F1093150188EF91E00E946E
:1044D0000B09082F809336068AEF91E00E940B09A2
:1044E0008093350687EF91E00E940B09182F809387
:1044F000340689EF91E00E940B0980933306115036
:104500008EE1189F102D1124185D0E94BD1E2FE012
:10451000029F202D112430E0A0E6BAEE0E94C335A0
:104520006C8B7D8B8E8B9F8B212F30E03D872C8772
:1045300022242394312C309137063F87809138060E
:10454000E82FEE0FFF0BE754FD4F459154915F8329
:104550004E83803351F58091A907082E000C990BEA
:10456000C09724E6289FA001299F500D1124485789
:104570005C4E8091AA07082E000C990BC0976AE048
:10458000689F9001699F300D1124240F351F809181
:10459000AB07082E000C990BC097D901A80FB91FC3
:1045A000BF83AE8380E30E940D090E94701B688B5D
:1045B000798B8A8B9B8B1A8604E1C02ED12C0E94AA
:1045C0007D0980936C068D3820F0B1E0B0936B06C6
:1045D00002C0893258F00E94701B60936706709386
:1045E00068068093690690936A0617C00E94701B44
:1045F00000916706109168062091690630916A065D
:10460000DC01CB01801B910BA20BB30B81379741CF
:10461000A105B10510F010926B060E94701B00916D
:104620003A0610913B0620913C0630913D06DC0194
:10463000CB01801B910BA20BB30B2C893D894E89BA
:104640005F89281739074A075B0798F48091360677
:10465000882379F00E94701B28EE33E040E050E0A0
:104660000E94A135643F71408105910510F40C94BE
:104670004C2F00913106109132064C855D85041750
:10468000150714F00C94522F80913406882311F4EE
:104690000C94522F0E94701B8090630690906406C9
:1046A000A0906506B0906606DC01CB0188199909D7
:1046B000AA09BB09893E9340A105B10510F40C94E9
:1046C000522F80916B06882311F40C94522F82E3B1
:1046D00090E00E94280B0C944730113009F069C01B
:1046E000E0906C06E09262060E94050B0E947D0934
:1046F000F82E80936C0620916E0630916F0690E044
:104700008217930708F4C90190936F0680936E0691
:1047100088E00E94841A892B79F484E690E00E9454
:10472000280B8091370690910201891302C081E025
:1047300001C08F5F809337068AE00E94841A892B1C
:1047400071F484E690E00E94280B80913706813056
:1047500019F48091020101C08150809337060091C5
:10476000370610E00754184FF8018081803340F479
:104770000E941B0B80937006D8018C9180933806A1
:1047800060913806862F062E000C990BFC01E85725
:10479000FD4FC490FC01EE0FFF1FE754FD4F059144
:1047A0001491A09061062F2D4091700681E00E9427
:1047B0005A13009116018EEF800F823008F024C149
:1047C00080916C06809362060E94050B0E947D0911
:1047D00080936C0620916E0630916F0690E08217F0
:1047E000930708F4C90190936F0680936E06F090CA
:1047F00038068F2D0E941B0BE82E80937006023026
:1048000011F00C942F3388E00E94841A892B09F050
:1048100041C084E690E00E94280B10E088E00E94EE
:10482000841A892B51F4153051F064E670E080E071
:1048300090E00E94361B1F5FF1CF153081F484E6B3
:1048400090E00E94280B88EF8F0D8093380688EF48
:104850008E0D8093700681E0809360060AC080917F
:104860006006811106C0F394F0923806E394E0925A
:10487000700680916006882339F088E00E94841ACF
:10488000019711F40C94273380917006803314F053
:10489000109270068AE00E94841A892B09F048C0A1
:1048A00084E690E00E94280B10E08AE00E94841ABF
:1048B000892B51F4153051F064E670E080E090E00F
:1048C0000E94361B1F5FF1CF153091F484E690E013
:1048D0000E94280B80913806885F8093380680916B
:1048E0007006885F8093700681E0809360060EC03A
:1048F0008091600681110AC08091380681508093B2
:104900003806809170068150809370068091600611
:10491000882339F08AE00E94841A019711F40C94DC
:104920002B338091700687FF03C08FE2809370065F
:104930008091380680331CF0805380933806809134
:10494000380687FF03C0805D8093380660910201BE
:1049500020913806022E000C330B9091610681E005
:10496000681710F40C944334E82FF0E0E754F84F44
:10497000408150E02417350721F481E080936106DF
:1049800025C08F5F90E0ECCF89E00E94841A892BCC
:1049900011F00C94033581E080935F0684E690E08B
:1049A0000E94280B81E0809373061092370688E2FC
:1049B00080932D0680915F06882311F40C94E233D6
:1049C00082E08093160181E0809339066091380679
:1049D000862F062E000C990BFC01E857FD4FC49062
:1049E000FC01EE0FFF1FE754FD4F05911491A090BD
:1049F0006106E090620620916C06409170068091FD
:104A000016010E945A13E4C3043019F0073009F06C
:104A1000DFC380916D06882349F010926D061091D6
:104A20003806812F0E940D0910932D0610916C06F7
:104A3000109362060E94050B0E947D094C018C8731
:104A400080936C06043071F4813560F099272091D1
:104A50006E0630916F062817390720F490936F0681
:104A600080936E06E0913806EE838E2FEE0F990B41
:104A7000FC01E857FD4FE491FC01EE0FFF1FE754E6
:104A8000FD4F8591949120910C0130910D01398752
:104A9000288740910E0150910F015B874A87509102
:104AA00070065E8781E08983073009F0198281E012
:104AB0008093E206EC858E2F90E0A0E0B0E09C01B0
:104AC000AD012150310941095109A9E2B0E00E942C
:104AD000963527EC30E040E050E00E947735290120
:104AE0003A01FFEF4F1A5F0A6F0A7F0A2090D8063B
:104AF0003090D9062E852223B9F0812F90E0A0E0D6
:104B0000B0E09C01AD012150310941095109A9E2F0
:104B1000B0E00E94963527EC30E040E050E00E9483
:104B200077352F5F2D8310C0E12CF12C04E310E0CA
:104B30002AE030E0A1014054510969E170E08EECB7
:104B400096E00E94201A1D82809101073E85381749
:104B500009F458C0C32ED12CCC0CDD1C56014BE1FE
:104B6000A40EB11C0EE110E0041915094091D806FD
:104B70005091D9064A525109E12CF12C22E030E043
:104B8000B5018EEC96E00E94201AA1014C5051090B
:104B900044195509EE24E394F12C820121E030E020
:104BA000B5018EEC96E00E94201A5E855E3298F484
:104BB0004091D8065091D90640545109E12CF12C6E
:104BC00004E310E022E030E0B601625E7F4F8EEC3D
:104BD00096E00E94201A4091D8065091D9064E5076
:104BE00051098A01041915098D81481B5109B60123
:104BF000675E7F4FEE24E394F12C95018EEC96E0F6
:104C00000E94CD048091FD069C85981750F0AE81DE
:104C1000A093FF06BE85B093FE068092FD064092EB
:104C2000050780910007EC85E81710F480920007D3
:104C3000E12CF12C0AE010E022E130E040E050E00D
:104C400060E070E08EEC96E00E94201AF981FF236C
:104C500069F14091D8065091D9064551510922E198
:104C600030E060E070E08EEC96E00E94201A8091C7
:104C7000D8069091D90644971092DB061092DA0676
:104C80009093DD068093DC068A859B850E941B132A
:104C90001092DB061092DA0682E090E09093DD0637
:104CA0008093DC06888599850E941B132E852F3200
:104CB00009F018C1E12CF12C0EE010E02AE030E000
:104CC00040E050E066E770E08EEC96E00E94201A2B
:104CD0008091FE06893118F0FBECCF2E01C0C12C6B
:104CE00080910507873018F487E08093050790913D
:104CF00005078AE2891B8093050782E08093E2061C
:104D0000E12CF12C04E110E025E130E047E150E036
:104D100060E070E08EEC96E00E94201A81E090E066
:104D20009093DF068093DE061092E1061092E00673
:104D30001092DB061092DA0688E190E09093DD068F
:104D40008093DC06E091FF06E83260F4F0E0E95D74
:104D5000FD4FE4916E2F70E080E090E040E10E9412
:104D6000DA120AC08CE40E9421138091FF0687703A
:104D700090E001960E942C1381E08093E206398135
:104D80003111B0C08091D8069091D9064797109202
:104D9000DB061092DA069093DD068093DC06E09144
:104DA000FF06F0E0EE0FFF1FEB53FE4F859194914D
:104DB0000E941B130C2C000CDD084091050750E0ED
:104DC0008091FE06B601680F711D680F711D6E5D42
:104DD0007F4FE12CF12C0FE010E02AE230E08EEC66
:104DE00096E00E94201A2091050730E04091FE06CF
:104DF000C601840F911D840F911D83969093DB064D
:104E00008093DA063093DD062093DC06E091FF06FE
:104E1000F0E0EE0FFF1FEB53FE4F859194910E943F
:104E20001B1383E695E00E94F2112091FD06822F6C
:104E300090E0A0E0B0E09C01AD01215031094109B2
:104E40005109A5E4B0E00E94963527EC30E040E03F
:104E500050E00E94773589010356110980910507BA
:104E600090E008962091FE06A601420F511D420FC8
:104E7000511D9A012D5D3F4F3093DB062093DA06DA
:104E80009093DD068093DC068DE20E942113882733
:104E90009927801B910B0E942C1384E595E00E94BA
:104EA000F2116091050770E06E5F7F4F8091FE0602
:104EB00090E00D9608E010E028E030E04DEB51E086
:104EC000880F991F0E9402201092FD061092FE0684
:104ED0001092FF060E94701168EE73E080E090E08F
:104EE0000E94361B0E9470114E85409301078091ED
:104EF00070068F3224F48F5F809370064AC110923F
:104F0000700680911601873009F043C180917106C7
:104F10009FEF980F9093710681113BC182E390E05F
:104F20000E94280B82E390E00E94280B82E390E02D
:104F30000E94280B60910E0170910F017093130174
:104F40006093120140910C0150910D014D375105B4
:104F500028F0509311014093100106C08EE591E0B6
:104F600090931101809310018091060190910701A7
:104F700090930B0180930A018091040190910501A7
:104F80008D37910510F48EE591E09093090180939F
:104F9000080180E00E943F1F8DE080931601B12C34
:104FA00092E0E92E2EE0A22E37E0932E40EA642E06
:104FB000712C0CE211E05EE5C52EDD24D39488E06F
:104FC0000E94841A892B29F484E690E00E94280B21
:104FD000BA948AE00E94841A892B29F484E690E02E
:104FE0000E94280BB394B7FC05C052E05B1524F473
:104FF000B12C02C082E0B82E40910C0150910D01FD
:1050000060910E0170910F018B2D0E943F1F89E06E
:105010000E94841A892BB9F581E0B81651F192E00B
:10502000B91651F190921601E09271067092130137
:10503000609212011093110100931001D0920F01A0
:10504000C0920E0170920D0160920C0170920B01E2
:1050500060920A011093090100930801D0920701A0
:10506000C092060170920501609204010E94D21E56
:1050700006C0A092160103C088E08093160184E662
:1050800090E00E94280B809116018D3009F497CF93
:105090008E30A1F56091120182E090E00E94090932
:1050A0006091130183E090E00E9409096091100172
:1050B00084E090E00E9409096091110185E090E090
:1050C0000E94090960910A0187E090E00E940909A5
:1050D00060910B0188E090E00E940909609108014D
:1050E00089E090E00E940909609109018AE090E05E
:1050F0000E94090983E0809316014BC0883009F0B3
:1051000048C085E090E00E940B09182F84E090E0F1
:105110000E940B09212F30E0322F2227282B3093B9
:1051200011012093100183E090E00E940B09182FD9
:1051300082E090E00E940B09212F30E0322F2227DD
:10514000282B309313012093120188E090E00E94F5
:105150000B09182F87E090E00E940B09212F30E007
:10516000322F2227282B30930B0120930A018AE04B
:1051700090E00E940B09182F89E090E00E940B0933
:10518000212F30E0322F2227282B30930901209342
:10519000080188E00E94841A892B81F484E690E05B
:1051A0000E94280B8FEF809314011092700681E00B
:1051B00080936D0610926F0610926E06E091700655
:1051C0000E2E000CFF0BE55EFC4FE491E0933806D9
:1051D000809116018A3009F059C082E390E00E9464
:1051E000280B80E00E943D1E89E00E94841A892BD2
:1051F000C1F3F0901501FA94E9E0EE2E18E006E014
:10520000A1E0FA1641F0B2E0FB1601F1F11005C081
:105210000093160102C0E09216018F2D0E943D1EE0
:1052200089E00E94841A892BA1F088E00E94841AE8
:10523000892B19F5FA9484E690E00E94280BE2E0AD
:10524000EF1514F1F7FEDCCF92E0F92E1093160162
:10525000E4CF89E00E94841A892B21F08091150106
:105260008093160184E690E00E94280B809116013D
:10527000883061F00E94650B09C08AE00E94841AA0
:10528000892BE9F6F394D7CFF12CC2CF8091160188
:10529000803111F40E94A20C809116018F3071F0C0
:1052A0001091380680912D0690E0212F012E000CE0
:1052B000330B8217930709F004C424C429EA37E0AA
:1052C0003A832983890172E7E72EFF24F394C7010B
:1052D0000E940B09D8018D938D01BFEFEB1AFB0AD9
:1052E000E8E7EE16E1E0FE0691F7CC24CA94DC2C48
:1052F00066246A94762CF1E0FC875FE1A52EB12C40
:1053000060E2262E312C29812A5F2D838FEA97E0D7
:1053100039E0380F388780903506909033065090EA
:10532000360650912C065A87809134068E8325E3E9
:1053300043E164E78CE10E94F4118C8563E00E94F4
:105340000B38492E9AE0499EA00111244B5E5F4F15
:10535000EE24E394F12C0AE010E025E530E06EE164
:1053600070E08EEC96E00E94201AAC85A3300CF021
:1053700070C081E090E0A11102C080E090E09093C5
:10538000E1068093E0069093DF068093DE06B092FC
:10539000DB06A092DA06E6E1F0E0F093DD06E093AA
:1053A000DC062E81E22FF0E0EE0FFF1FE058FD4FEC
:1053B0006591749186E097E00E945A3586E097E007
:1053C0000E94F21181E090E031E0431202C080E0DF
:1053D00090E09093E1068093E0069093DF0680933F
:1053E000DE06B092DB06A092DA063092DD0620924D
:1053F000DC06E52DF0E0EE0FFF1FE858FD4F65914C
:10540000749186E097E00E945A3586E097E00E940A
:10541000F21181E090E042E0441202C080E090E0AE
:105420009093E1068093E0069093DF068093DE067A
:10543000B092DB06A092DA068AE290E09093DD0655
:105440008093DC06E82DF0E0EE0FFF1FEC58FD4FD7
:10545000B6C19C8596300CF04BC15C2C81E090E08D
:10546000411002C080E090E09093E1068093E00656
:105470009093DF068093DE06B092DB06A092DA06F8
:10548000A6E1B0E0B093DD06A093DC06E92DF0E0E4
:10549000EE0FFF1FE059FD4F6591749186E097E094
:1054A0000E945A3586E097E00E94F21181E090E078
:1054B000B1E04B1202C080E090E09093E10680934F
:1054C000E0069093DF068093DE0657FCC6C0E12C11
:1054D000F12C0AE010E025E530E04FE150E06EE10C
:1054E00070E08EEC96E00E94201A81E090E09093AC
:1054F000E1068093E0069093DF068093DE06B0928B
:10550000DB06A092DA063092DD062092DC0687E602
:1055100095E00E94F21109E010E026E230E04FE150
:1055200050E068E470E08EEC96E00E94201A852C32
:10553000052C000C9908E52DF6E0EF02B0011124CE
:10554000685B7F4FEE24E394F12C27E030E04FE1DD
:1055500050E08EEC96E00E94201AB9EAEB2EB7E0FC
:10556000FB2E00E010E081E090E00815190511F431
:1055700080E090E09093E1068093E0069093DF0650
:105580008093DE06D7018D917D010E9421130F5F6C
:105590001F4F0630110539F7562C81E090E0B2E03C
:1055A0004B1202C080E090E09093E1068093E00609
:1055B0009093DF068093DE0657FC81C0E12CF12C2E
:1055C0000AE010E025E530E049E250E06EE170E0ED
:1055D0008EEC96E00E94201A81E090E09093E10624
:1055E0008093E0069093DF068093DE06B092DB06A0
:1055F000A092DA062AE230E03093DD062093DC0642
:105600008FE695E00E94F21109E010E026E230E01A
:1056100049E250E06CE370E08EEC96E00E94201AC4
:10562000852C052C000C9908352D46E03402B0017C
:105630001124645C7F4FEE24E394F12C27E030E0EA
:1056400049E250E08EEC96E00E94201AFFEA4F2ECD
:10565000F7E05F2E00E010E02AC0B092DB06A092D7
:10566000DA063092DD062092DC0687E695E00E949D
:10567000F21109EA17E0F80181918F010E942113CC
:10568000FD81F013F8CF88CF9093E1068093E00678
:105690009093DF068093DE06D2018D912D010E944A
:1056A00021130F5F1F4F0930110509F492C081E0EB
:1056B00090E00815190541F780E090E0E5CFB09241
:1056C000DB06A092DA06EAE2F0E0F093DD06E09372
:1056D000DC068FE695E00E94F2110FEA17E0D80190
:1056E0008D918D010E942113B885B013F8CF71C040
:1056F00081E090E0411002C080E090E09093E106EC
:105700008093E0069093DF068093DE06B092DB067E
:10571000A092DA06E6E1F0E0F093DD06E093DC0625
:105720002A85E22FF0E0EE0FFF1FE659FD4F65914D
:10573000749186E097E00E945A3586E097E00E94D7
:10574000F21181E090E031E0431202C080E090E08D
:105750009093E1068093E0069093DF068093DE0647
:10576000B092DB06A092DA063092DD062092DC06CB
:10577000E6E6F2E06591749186E097E00E945A3582
:1057800086E097E00E94F21181E090E042E044124E
:1057900002C080E090E09093E1068093E006909351
:1057A000DF068093DE06B092DB06A092DA068AE27C
:1057B00090E09093DD068093DC06E4E6F2E06591EC
:1057C000749186E097E00E945A3586E097E00E9447
:1057D000F2110E94701189E00E94841A892B09F04D
:1057E000C5C084E690E00E94280BEC858E2FEE0F5A
:1057F000990BAA0BBB0B8930910510F00C94103556
:10580000FC01EC5CFF4F0C94173882E390E00E949F
:10581000280B82E390E00E94280B82E390E00E9434
:10582000280B87E09BC0809134068F5F843018F48A
:105830008093340602C0109234066091340687EFDC
:1058400091E00EC0809136068F5F843018F480930B
:10585000360602C0109236066091360688EF91E057
:105860000E94090958CD809135068F5F823018F467
:105870008093350602C010923506609135068AEF96
:1058800091E0EECF809133068F5F823019F08093E4
:10589000330602C0109233066091330689EF91E01F
:1058A000DFCFFFEFCF1ADF0A23E0C216D10449F0A1
:1058B00036E0C316D1040CF42ECDCC24CA94DC2CD3
:1058C0002ACD44E0C42ED12C8091A907082E000CCB
:1058D000990BC09724E6289FA001299F500D112401
:1058E0008091AA07082E000C990BC0976AE0689F68
:1058F0009001699F300D1124240F351F8091AB0753
:10590000082E000C990BC097280F391F2C3241E04C
:10591000340708F0ABC083E38093A90780E380934A
:10592000AA07AEC05FEF651A750A89E068167104B0
:105930000CF4F1CC66246A94762CEDCC80912C0684
:105940008F5F833018F480932C0602C010922C06CF
:1059500060912C0686EF91E083CF88E0809316015A
:105960000FEA17E025E6E22EF12C8DC088E00E94B8
:10597000841A892BB1F584E690E00E94280B9FEFF2
:105980006916790641F4AFEFCA16DA0621F4BC8530
:10599000B150BC8764C0EC85E53051F4F301E155AA
:1059A000F84F80818F5F8E370CF080E28083B3CC1C
:1059B000FC85F43011F00C941035F601E755F84FE2
:1059C00080818F5F808324E0C216D10429F08A335E
:1059D0000CF4A1CC80E3EACF8B350CF49CCC81E4B1
:1059E0003BC08AE00E94841A892B11F00C94103578
:1059F00084E690E00E94280B3FEF6316730641F4A3
:105A00004FEFC416D40621F45C855F5F5C8727C026
:105A10008C85853049F4F301E155F84F8081815040
:105A2000803224F68DE7C2CF9C85943011F00C941F
:105A30001035F601E755F84F808181508083A4E04E
:105A4000CA16D10429F080330CF065CC89E3AECFBF
:105A500087340CF060CC8AE58093AD075CCCBC85C4
:105A6000B93014F00C9415350C940735263E3340AC
:105A700008F451CC89E38093A9078093AA0787E3B0
:105A80008093AB0748CCD8016D918D01C7010E946E
:105A90000909BFEFEB1AFB0AEFE6EE16F10499F7DE
:105AA00002E711E0A981BA816D91BA83A983C80187
:105AB0000E9409090F5F1F4F0837B1E01B0791F7DC
:105AC000EFCB812F0E940D0910932D060E94701BB1
:105AD000609328067093290680932A0690932B06DC
:105AE00080910001882371F01092000182E390E020
:105AF0000E94280B82E390E00E94280B82E390E052
:105B00000E94280B80E090E0892B11F40C948021F6
:105B10000E9400000C948021883019F480E10C94DC
:105B2000DB2186E00C94DB219D819330C1F02CF4C5
:105B3000913059F0923059F005C0AD81A43099F000
:105B4000A530A1F03092160114C082E010C083E0AD
:105B50008093160130927406109273060AC0B4E066
:105B6000B093160106C02092160103C088E080930E
:105B7000160126E34AE068E688E10E94F411EE246B
:105B8000E394F12C0AE010E02DE430E046E150E02F
:105B90006AE170E08EEC96E00E94201AED81E1113E
:105BA00017C0F2016591749186E097E00E945A3522
:105BB000F601659174918AE197E00E945A35F501EA
:105BC000659174918EE297E00E945A35F30182C08C
:105BD000FD81F130B9F4F6016591749186E097E0AA
:105BE0000E945A35F501659174918AE197E00E940F
:105BF0005A35F301659174918EE297E00E945A350F
:105C0000F40168C02D812230C1F4F50165917491D1
:105C100086E097E00E945A35F301659174918AE11C
:105C200097E00E945A35F401659174918EE297E0F5
:105C30000E945A35E0E6F2E04DC03D813330C1F4B8
:105C4000F3016591749186E097E00E945A35F40162
:105C5000659174918AE197E00E945A35E0E6F2E09E
:105C6000659174918EE297E00E945A35F20132C03C
:105C70004D814430C1F4F4016591749186E097E060
:105C80000E945A35E0E6F2E0659174918AE197E06E
:105C90000E945A35F201659174918EE297E00E945C
:105CA0005A35F60117C0E0E6F2E06591749186E09E
:105CB00097E00E945A35F201659174918AE197E06C
:105CC0000E945A35F601659174918EE297E00E9428
:105CD0005A35F5016591749182E497E00E945A3536
:105CE0001092E1061092E0061092DF061092DE0696
:105CF0008091D6069091D7068854910997FD019618
:105D0000959587959093DB068093DA0688E190E07D
:105D10009093DD068093DC068AE197E00E94F21101
:105D200081E090E09093E1068093E0069093DF0697
:105D30008093DE068091D6069091D706885491090B
:105D400097FD0196959587959093DB068093DA06EB
:105D5000AEE0B0E0B093DD06A093DC0686E097E00D
:105D60000E94F2118091D6069091D706885491092D
:105D700097FD0196959587959093DB068093DA06BB
:105D8000E2E2F0E0F093DD06E093DC068EE297E0DD
:105D90000E94F2118091D6069091D70688549109FD
:105DA00097FD0196959587959093DB068093DA068B
:105DB0002CE230E03093DD062093DC0682E497E0AD
:105DC0000E94F2110E94701189E00E94841A892BAE
:105DD00079F489E00E94841A892B21F080911501C1
:105DE0008093160184E690E00E94280B0C94DD213C
:105DF00088E00E94841A892B41F484E690E00E9496
:105E0000280B3D8131503D8313C08AE00E94841AE3
:105E1000892B71F484E690E00E94280B4D814F5F3E
:105E20004D83463011F00C94CF211D820C94CF216C
:105E3000ED81E7FD02C00C94CF21F5E0FD830C94C9
:105E4000CF214AEA50E050931301409312018EE5AE
:105E500091E0909311018093100190930F01809332
:105E60000E0120EA30E030930D0120930C01509395
:105E70000B0140930A0190930901809308019093CC
:105E8000070180930601309305012093040182E00D
:105E9000809371060C94032282E390E00E94280B09
:105EA0000C94392380912F06909130062C853D85E6
:105EB00082179307ECF4809134068823C9F00E947E
:105EC000701B8090630690906406A0906506B09069
:105ED0006606DC01CB0188199909AA09BB09893E2C
:105EE0009340A105B10520F080916B068111CFC0D0
:105EF000F0913306F88F209138062E8F622F022EF4
:105F0000000C770BFB01E857FD4FF490B0902E0684
:105F1000309134063D8380902F06098340916C06B2
:105F2000498F5091010158878091020728130E94E0
:105F3000BD1E8FEFF81651F195E09093E206309276
:105F4000E1062092E0063092DF062092DE061092F3
:105F5000DB061092DA06AFE0B0E0B093DD06A09366
:105F6000DC06BE8DB83240F46F2D70E080E090E02A
:105F700040E10E94DA1227C08CE40E9421138E8D2A
:105F8000877090E001960E942C131DC0E5E0E0931D
:105F9000E2063092E1062092E0063092DF0620927F
:105FA000DE061092DB061092DA062FE030E0309326
:105FB000DD062093DC068091AD070E9421138091BD
:105FC000AE070E94211331E03093E2061092DF0603
:105FD0001092DE063092E1062092E006EE24E39471
:105FE000F12C09E010E027E030E040E050E060E014
:105FF00070E08EEC96E00E94201A3092DB06209230
:10600000DA063092DD062092DC0680E595E00E94FB
:10601000F2114091D8065091D9064950510927E014
:1060200030E060E070E08EEC96E00E94201A8091F3
:10603000D8069091D90608973092DB062092DA06AE
:106040009093DD068093DC0682E595E00E94F211D4
:10605000E12CF12C02E310E027E330E042E150E0D4
:1060600066E470E08EEC96E00E94201ABB20F1F00E
:106070000E94701B20E233E040E050E00E94A13516
:10608000603971408105910508F42AC20FC082E38E
:1060900090E00E94280B0E94701B6093630670932F
:1060A0006406809365069093660622CF3092E106DF
:1060B0002092E0063092DF062092DE0682E0809396
:1060C000E20606E410E01093DB060093DA064CE1EA
:1060D00050E05093DD064093DC068E819F810E9444
:1060E0001B131093DB060093DA0682E190E0909395
:1060F000DD068093DC0651E05093E2068FEA97E0DC
:106100000E94F2119EE18D818150899F802D112482
:10611000885D8E87912CA12CB12C51E0851A9108B5
:10612000A108B108A4E7B0E0A50194010E9496354A
:1061300027EC30E040E050E00E94773529013A0139
:1061400083E0480E511C611C711C27E730E02419C4
:106150003509B201695F7F4FE12CF12C09E010E0B5
:1061600040E050E08EEC96E00E94201A9885923034
:1061700069F4EE24E394F12C920140E050E067E0F2
:1061800070E08EEC96E00E94201A1AC0E12CF12CEF
:1061900009E010E027E730E040E050E067E070E021
:1061A0008EEC96E00E94201AEE24E394F12C9201EA
:1061B00040E050E067E070E08EEC96E00E947E04E4
:1061C000A9810A2F10E020E030E028013901B1E078
:1061D0004B1A510861087108A4E7B0E0A3019201CD
:1061E0000E94963527EC30E040E050E00E94773581
:1061F000DA01C9010396A11DB11D89839A83AB837E
:10620000BC8327E730E0281B390B4091D80650911A
:10621000D9064950510969817A81695F7F4FE12C24
:10622000F12C09E010E08EEC96E00E94201A4091DB
:10623000D8065091D906988549505109913061F49A
:10624000EE24E394F12C29813A8167E070E08EEC32
:1062500096E00E94201A1DC0E12CF12C09E010E00C
:1062600027E730E067E070E08EEC96E00E94201AAD
:106270004091D8065091D90649505109EE24E39433
:10628000F12C29813A8167E070E08EEC96E00E9463
:106290007E041092DF061092DE063092E106209214
:1062A000E006A88DA1114FC0A3E6B0E0A3019201C2
:1062B0000E94963527EC30E040E050E00E947735B0
:1062C000122FA3E6B0E0A50194010E94963527ECB9
:1062D00030E040E050E00E94773549015A01BFEFBD
:1062E0008B1A9B0AAB0ABB0AD092DB06C092DA0675
:1062F000E8E3F0E0F093DD06E093DC0661E0610F97
:10630000653608F064E670E080E090E04AE00E94C4
:10631000DA1285E20E942113D092DB06C092DA06DF
:106320003092DD062092DC06882D853608F084E662
:10633000682F70E080E090E04AE00E94DA1285E287
:106340000E94211350C0A5E4B0E0A30192010E9475
:10635000963527EC30E040E050E00E947735290187
:106360003A01A5E4B0E0A50194010E94963527EC1E
:1063700030E040E050E00E947735D092DB06C092DA
:10638000DA0688E390E09093DD068093DC068DE2E8
:106390002A8F3B8F4D8F5C8F0E942113C201835641
:1063A00091099195819591090E942C1384E595E0BE
:1063B0000E94F211D092DB06C092DA063092DD061E
:1063C0002092DC068DE20E9421132A8D3B8DC901AB
:1063D000835691099195819591090E942C1384E52A
:1063E00095E00E94F211998DAE859A1780F5BD81D6
:1063F000BB2369F10E94701B2AEF30E040E050E0BF
:106400000E94A13521E030E06D37710581059105CD
:1064100010F020E030E03093DF062093DE0610928B
:10642000E1061092E0068091D8069091D906439734
:1064300020E430E03093DB062093DA069093DD060B
:106440008093DC0688E595E00E94F21112C040912D
:10645000D8065091D90643515109E12CF12C09E09D
:1064600010E02CE330E060E470E08EEC96E00E94F7
:10647000201A0E947011EE8DE09302070E946B10AB
:10648000082F0E94701BDC01CB01288939894A89B9
:106490005B89821B930BA40BB50B81319742A1053D
:1064A000B10550F04A85442319F051E05A8704C0E1
:1064B00080913506882309F18AE00E94841A0197A9
:1064C00039F588E00E94841A019711F589E00E944D
:1064D000841A0197E9F48F8D08131AC00C94DF22F7
:1064E00000E110E020E130E04DE951E067E170E0CB
:1064F00080E590E00E94022005CE81E080932E0688
:1065000015E082E390E00E94280B1150D1F7CDCF27
:1065100080912E06811129C088E00E94841A892B5F
:1065200081F484E690E00E94280B809137069091D8
:106530000201891303C01092370603C08F5F809356
:1065400037068AE00E94841A892B01F584E690E0E0
:106550000E94280B80913706811103C080910201AF
:1065600001C081508093370611C0D12C89E00E9470
:10657000841A892B61F495E0D91649F064E670E03D
:1065800080E090E00E94361BD394F0CFD12C809114
:106590003706AF8DA01748F490910201891303C00C
:1065A000109237060DC08F5F09C0BF8D0B1748F4DE
:1065B000811103C08091020101C081508093370690
:1065C0000F8F90913706092F10E00754184FF801EC
:1065D0008081813358F4FF859F1741F00E941B0B87
:1065E00080937006D8018C918093380610913806FC
:1065F000412F012E000C550B20912D0630E0421743
:10660000530739F0812F0E940D090E947D09809364
:106610006C0610926B0610932D0689E00E94841A76
:10662000019711F40C949B22B5E0DB1203C00E9489
:10663000A20C04C08091150180931601109263068C
:106640001092640610926506109266065BCA10925C
:1066500060060C944424109260060C94912480915E
:10666000730681110C94DA2410925F068FEF8093E9
:106670005E0646E5642E46E0742E56E4852E56E00E
:10668000952E4EE356E0B401C301EEE4F6E028E0B7
:106690002E0F1192DC011D92CD01DB011D92BD0177
:1066A000DA011D92AD012E13F4CF32E0532EF12CFE
:1066B000DD24D3941092700640917006E42F042ECE
:1066C000000CFF0BE55EFC4FB490B09238068B2DAA
:1066D0004D8F0E940D0962E370E080E090E00E941F
:1066E000361BE0906C06E09262060E94050B0E9449
:1066F0007D0980936C06E0916E06F0916F06682F1D
:1067000070E04D8D6E177F0708F4BF0170936F0620
:1067100060936E066B2D0B2C000C770BFB01E8577A
:10672000FD4FC490FB01EE0FFF1FE754FD4F059195
:106730001491A0906106282F6B2D83E00E945A13BC
:1067400020916C06213A08F17091020130913806CF
:10675000432F032E000C550B60E0E62FF0E0E754CA
:10676000F84F808190E04817590721F06F5F761746
:10677000A0F78DC08F2D90E0FC01EA5BF94F3083CC
:10678000FC01E25CF94F2083F394109170061F5FC7
:106790001093700689E00E94841A892B19F4D09214
:1067A0005F0602C010925F0610330CF0BDC089E096
:1067B0000E94841A019709F0B7C080915F06811189
:1067C000B3C07ACF10915E061F3FB9F481E00E94FA
:1067D0009B126CED75E080E090E00E94361B82E039
:1067E0008093160181E0809339068EE190E00E944B
:1067F0000B09809337060C94E6240E94050B0E9437
:106800007D0980936C0688E00E94841A892BA9F484
:1068100084E690E00E94280B80913706482F50E0D4
:10682000212F012E000C330B4217530719F410923D
:10683000370603C08F5F809337068AE00E94841A70
:10684000892B71F484E690E00E94280B8091370632
:10685000811103C01093370603C08150809337061F
:10686000E0913706F0E0EA5AF94F1081103310F04A
:106870000C94E624812F0E941B0B809370061093CA
:1068800038060C94E624909361060C94E6248091DB
:106890005E06873054F48F5F80935E06082E000CEE
:1068A000990BFC01EA5AF94F09C0082E000C990B0C
:1068B000FC01EA5AF94F4081421728F42083FC0179
:1068C000E25BF94F308350915E06E0E05E170CF416
:1068D0005CCF61E06E0F462F0E2E000CFF0BCF0138
:1068E0008A5A994F9F01225B394F59015417D4F0AE
:1068F000A42F042E000CBB0B9D012A5A394FF9011D
:106900001081FC017081711758F4F5010081A25BC0
:10691000B94FEC90E0820C93DC011C93F901708379
:106920004F5FE4CFE62FD2CF10915E061F3F29F4D0
:1069300089E00E94841A019721F060E02F2D30E059
:1069400026C0F1E05F16C9F35524539480915F0689
:106950008111F3CFAFCEAC01425C594FDA010C91FB
:10696000D501CC90C01658F4E0808A5B994FDC01C9
:10697000DC90D082EC92D5010C93DA01CC927F5F4F
:10698000872F072E000C990B8217930724F3E62F0D
:10699000062E000CFF0BE217F3074CF46F5F762F07
:1069A000AF01425C594F5A01EA5BF94FE9CF1F0D25
:1069B00010935E0617301CF087E080935E064091CE
:1069C0005E06042E000C550B60E02A5A394F862FC4
:1069D00090E04817590754F0F901E80FF91FDC015E
:1069E000A25BB94F8C9180836F5FF1CFE6E5F6E053
:1069F0008E2F86198F1510F00C94C424D4018D911C
:106A00004D018193F5CF10925F060C94D2249C85A2
:106A100097FD02C00C948B2948E04C870C948B297D
:106A2000AC85A93014F40C948B291C860C948B290A
:106A3000E2ECF6E01382128288EE93E0A0E0B0E090
:106A400084839583A683B7838CE295E091838083CA
:106A5000EEECF6E01382128220E830E035832483E6
:106A600080E490E0978386833187208793878287AD
:106A7000158A158614861786168681E0848B2FEF7B
:106A80003FEF338B228B318B208B868B178A118EB5
:106A9000108E8CE395E0918380838FEF848F80A3A9
:106AA000868F858F97E0978FECEFF6E0858387835D
:106AB00010820895FB01DC0105900D920020E1F7A2
:106AC0000895F999FECF92BD81BDF89A992780B5B6
:106AD0000895262FF999FECF1FBA92BD81BD20BD22
:106AE0000FB6F894FA9AF99A0FBE01960895052EFA
:106AF00097FB1EF400940E948E3557FD07D00E942C
:106B0000A13507FC03D04EF40C948E35509540957A
:106B1000309521953F4F4F4F5F4F08959095809549
:106B2000709561957F4F8F4F9F4F08950E94C33599
:106B3000A59F900DB49F900DA49F800D911D1124D1
:106B40000895A1E21A2EAA1BBB1BFD010DC0AA1FAE
:106B5000BB1FEE1FFF1FA217B307E407F50720F0C6
:106B6000A21BB30BE40BF50B661F771F881F991F41
:106B70001A9469F760957095809590959B01AC018A
:106B8000BD01CF010895A29FB001B39FC001A39F93
:106B9000700D811D1124911DB29F700D811D112456
:106BA000911D08955058BB27AA270E94EA350C94DE
:106BB0003B370E942D3738F00E94343720F039F4EB
:106BC0009F3F19F426F40C942A370EF4E095E7FB66
:106BD0000C942437E92F0E944C3758F3BA176207F8
:106BE00073078407950720F079F4A6F50C946E37A7
:106BF0000EF4E0950B2EBA2FA02D0B01B9019001D8
:106C00000C01CA01A0011124FF27591B99F0593F1B
:106C100050F4503E68F11A16F040A22F232F342F63
:106C20004427585FF3CF469537952795A795F040B1
:106C30005395C9F77EF41F16BA0B620B730B840BC6
:106C4000BAF09150A1F0FF0FBB1F661F771F881F7E
:106C5000C2F70EC0BA0F621F731F841F48F48795D6
:106C600077956795B795F7959E3F08F0B0CF9395C8
:106C7000880F08F09927EE0F9795879508950E9441
:106C800053360C943B370E94343758F00E942D370E
:106C900040F029F45F3F29F00C94243751110C94F3
:106CA0006F370C942A370E944C3768F39923B1F35D
:106CB000552391F3951B550BBB27AA276217730722
:106CC000840738F09F5F5F4F220F331F441FAA1FB6
:106CD000A9F335D00E2E3AF0E0E832D09150504072
:106CE000E695001CCAF72BD0FE2F29D0660F771F20
:106CF000881FBB1F261737074807AB07B0E809F006
:106D0000BB0B802DBF01FF2793585F4F3AF09E3F8A
:106D1000510578F00C9424370C946F375F3FE4F3FF
:106D2000983ED4F3869577956795B795F7959F5FCD
:106D3000C9F7880F911D9695879597F90895E1E019
:106D4000660F771F881FBB1F621773078407BA0778
:106D500020F0621B730B840BBA0BEE1F88F7E095D3
:106D600008950E94B8366894B1110C946F37089555
:106D70000E94543788F09F5798F0B92F9927B75140
:106D8000B0F0E1F0660F771F881F991F1AF0BA95CF
:106D9000C9F714C0B13091F00E946E37B1E0089588
:106DA0000C946E37672F782F8827B85F39F0B93F7A
:106DB000CCF3869577956795B395D9F73EF4909582
:106DC0008095709561957F4F8F4F9F4F0895E89400
:106DD00009C097FB3EF490958095709561957F4F23
:106DE0008F4F9F4F9923A9F0F92F96E9BB279395D1
:106DF000F695879577956795B795F111F8CFFAF4E1
:106E0000BB0F11F460FF1BC06F5F7F4F8F4F9F4F11
:106E100016C0882311F096E911C0772321F09EE86F
:106E2000872F762F05C0662371F096E8862F70E0D5
:106E300060E02AF09A95660F771F881FDAF7880FAF
:106E40009695879597F9089597F99F6780E870E080
:106E500060E008959FEF80EC089500240A941616D0
:106E6000170618060906089500240A941216130638
:106E7000140605060895092E0394000C11F48823C6
:106E800052F0BB0F40F4BF2B11F460FF04C06F5FE2
:106E90007F4F8F4F9F4F089557FD9058440F551FB8
:106EA00059F05F3F71F04795880F97FB991F61F08C
:106EB0009F3F79F087950895121613061406551F03
:106EC000F2CF4695F1DF08C0161617061806991F6F
:106ED000F1CF86957105610508940895E894BB2764
:106EE00066277727CB0197F908950E94E73708F4C2
:106EF0008FEF08950E948D370C943B370E942D37F9
:106F000038F00E94343720F0952311F00C94243788
:106F10000C942A3711240C946F370E944C3770F36D
:106F2000959FC1F3950F50E0551F629FF001729F2E
:106F3000BB27F00DB11D639FAA27F00DB11DAA1F3D
:106F4000649F6627B00DA11D661F829F2227B00D8A
:106F5000A11D621F739FB00DA11D621F839FA00D15
:106F6000611D221F749F3327A00D611D231F849F65
:106F7000600D211D822F762F6A2F11249F575040BC
:106F80009AF0F1F088234AF0EE0FFF1FBB1F661F37
:106F9000771F881F91505040A9F79E3F510580F000
:106FA0000C9424370C946F375F3FE4F3983ED4F38E
:106FB000869577956795B795F795E7959F5FC1F7A4
:106FC000FE2B880F911D9695879597F90895990F37
:106FD0000008550FAA0BE0E8FEEF16161706E807A3
:106FE000F907C0F012161306E407F50798F0621BC4
:106FF000730B840B950B39F40A2661F0232B242B99
:10700000252B21F408950A2609F4A140A6958FEFB7
:10701000811D811D0895991B79E004C0991F961761
:1070200008F0961B881F7A95C9F780950895EE0F92
:10703000FF1F0590F491E02D099481E090E0F89411
:107040000C942938FB01DC0101900D920020E1F73E
:067050000895F894FFCF43
:10705600010108505E01A0005E01A0005E01A000D3
:107066005E01A00004030300000000000000000011
:10707600000000000000000000000000000000000A
:1070860000000000000000000000000000000000FA
:1070960000000000000000000000000080808080EA
:1070A600C0C0C0C0C0C0C0C0C0C0C0C0C0C0C0C0DA
:1070B60080808080000000000000000000000000CA
:1070C60000000000000000000000000000000000BA
:1070D60000000000000000000000000000000000AA
:1070E600000000000000000000000000000000009A
:1070F600000000000000000000000000000000008A
:10710600000000000000000000000080C0C0E0E0B9
:10711600F0F0F8F8FCFCFE7E7E3F3F3F1F1F1F0F7E
:107126000F0F0F8F8F8787878787878F8F0F0F0F99
:107136001F1F1F1F3F3F3F7E7EFEFCFCF8F8F0F04E
:10714600E0E0C0C080000000000000000000000079
:107156000000000000000000000000000000000029
:107166000000000000000000000000000000000019
:107176000000000000000000000000000000000009
:10718600000080C0E0F0F8FCFEFF7F3F1F1F0F07E6
:1071960007030301000000000080E0F0F8FCFCFE9D
:1071A600FF7F3F3F1F1F1F1F1F1F1F1F3F3F7FFFE9
:1071B600FEFCFCF8F0E0800000000001010303077C
:1071C600070F1F3F3F7FFEFEFCF8F0E0C080000087
:1071D60000000000000000000000000000000000A9
:1071E6000000000000000000000000000000000099
:1071F6000000000000000000000000C0E0F0F8FC05
:10720600FEFF7F3F1F0F07030100FCFC0C8C8C8CDC
:107216008C8C8C0C0C0000F8FFFFFFFFFF0F0301A6
:107226000000FCFC1C1C1C1C1C1C1C1CFCF800008C
:1072360001030FFFFFFFFFFFF8000C3CF8E08000A2
:10724600000080E0F83C0C0103070F1F3F7FFFFEA4
:10725600FCF8F0E0C00000000000000000000000A4
:107266000000000000000000000000000000000018
:10727600000000000000000000000003070F1F3F91
:107286007FFFFEFCF8F0E0C080007F7F0001010177
:10729600010101000000001FFFFFFFFFFFF0C0809B
:1072A60000007F7F000707070707070703010000A5
:1072B60080C0F0FFFFFFFF7F1F00000000071F7E5A
:1072C600783E0F0300000080C0E0F0F8FCFEFF7F70
:1072D6003F1F0F0703000000000000000000000031
:1072E6000000000000000000000000000000000098
:1072F6000000000000000000000000000000000088
:1073060000000103070F1F3F7FFFFEFCF8F8F0E0C7
:10731600E0C0C080000000000001070F1F3F3F7F54
:10732600FFFEFCFCF8F8F8F8F8F8F8F8FCFCFEFFAD
:107336007F3F3F1F0F0701000000008080C0C0E0B4
:10734600E0F0F8FCFCFE7F7F3F1F0F070301000003
:107356000000000000000000000000000000000027
:107366000000000000000000000000000000000017
:107376000000000000000000000000000000000007
:1073860000000000000000000000000103030707E2
:107396000F0F1F1F3F3F7F7E7EFCFCFCF8F8F8F8BE
:1073A600F0F0F0F1F1F1E1E1E1E1F1F1F1F0F0F00D
:1073B600F8F8F8F8FCFCFC7E7E7F3F3F1F1F0F0F9E
:1073C60007070303010000000000000000000000A2
:1073D60000000000000000000000000000000000A7
:1073E6000000000000000000000000000000000097
:1073F6000000000000000000000000000000000087
:107406000000000000000000000000000000000076
:107416000000000000000000000000000101010162
:107426000303030303030303030303030303030326
:107436000101010100000000000000000000000042
:107446000000000000000000000000000000000036
:107456000000000000000000000000000000000026
:107466000000000000000001000103070F1F3F7F1E
:107476000080C0E0F0F8FCFE00000000551725175C
:107486001D170E170017FF16000000002B195416C3
:107496002D08CD047705D1067E04201A021A84171A
:1074A6004200410064426D004C4F57205349474EFD
:1074B600414C004D687A004E45575F463A350053B9
:1074C60049474E3A00465552494F555300333632D6
:1074D600204C310043414E27542044454C455445E9
:1074E60000492043414E27542046494E4400544803
:1074F6004953204348414E4E454C0053415645445E
:107506000046004300204C4F434B00554E4C4F4322
:107516004B00205341564520005341564500434FEA
:107526004D504C45544521004D487A00353336328E
:107536000035383030003539343500424553540073
:107546002C0052452D43414C49425241544500536B
:107556004156452026204558495400574F524B491D
:107566004E47004D414E55414C00534D415254003B
:08757600534541524348000057
:00000001FF
